S00F0000746563776172652E737265632A
S3150800280000000120F5C900088D5200089B520008F7
S31508002810A9520008B7520008C55200080000000077
S31508002820000000000000000000000000E1C40008ED
S31508002830D35200080000000081C50008D5520008E0
S3150800284045CA000845CA000845CA000845CA00081E
S3150800285045CA000845CA000845CA000845CA00080E
S3150800286045CA000845CA000845CA000845CA0008FE
S31508002870ED520008FD52000845CA000845CA00087E
S3150800288045CA000845CA00080D5300081D5300082C
S315080028902D5300083D5300084D53000845CA00084B
S315080028A045CA000845CA000845CA000845CA0008BE
S315080028B045CA0008000000000000000045CA0008DC
S315080028C045CA000800000000000000005D5300082B
S315080028D00000000045CA000845CA000800000000BC
S315080028E045CA000845CA00080000000000000000AC
S315080028F000000000000000000000000000000000CA
S3150800290000000000000000000000000045CA0008A2
S31508002910000000000000000045CA000845CA00087B
S3150800292045CA000845CA00086D53000845CA00088C
S3150800293045CA000800000000000000000000000072
S3150800294045CA000845CA000845CA000845CA00081D
S3150800295045CA000845CA000845CA000845CA00080D
S3150800296045CA000845CA000845CA00080000000014
S3150800297045CA000845CA000800000000000000001B
S3150800298045CA000845CA000845CA00082255AAEEE5
S3150800299010B5054C237833B9044B13B10448AFF38B
S315080029A000800123237010BD1801002000000000DC
S315080029B018CC000808B5034B1BB103490348AFF30D
S315080029C0008008BD000000001C01002018CC00088B
S315080029D081F0004102E000BF83F0004330B54FEAC2
S315080029E041044FEA430594EA050F08BF90EA020F2F
S315080029F01FBF54EA000C55EA020C7FEA645C7FEAC2
S31508002A00655C00F0E2804FEA5454D4EB5555B8BFE4
S31508002A106D420CDD2C4480EA020281EA030382EA55
S31508002A20000083EA010180EA020281EA0303362DE7
S31508002A3088BF30BD11F0004F4FEA01314FF4801CBA
S31508002A404CEA113102D0404261EB410113F0004FCC
S31508002A504FEA03334CEA133302D0524263EB430383
S31508002A6094EA050F00F0A780A4F10104D5F1200E21
S31508002A700DDB02FA0EFC22FA05F2801841F100017C
S31508002A8003FA0EF2801843FA05F359410EE0A5F150
S31508002A9020050EF1200E012A03FA0EFC28BF4CF081
S31508002AA0020C43FA05F3C01851EBE37101F0004537
S31508002AB007D54FF0000EDCF1000C7EEB00006EEB44
S31508002AC00101B1F5801F1BD3B1F5001F0CD34908CE
S31508002AD05FEA30004FEA3C0C04F101044FEA445225
S31508002AE012F5800F80F09A80BCF1004F08BF5FEAAC
S31508002AF0500C50F1000041EB045141EA050130BD8C
S31508002B005FEA4C0C404141EB0101013C28BFB1F59D
S31508002B10801FE9D291F0000F04BF01460020B1FAE8
S31508002B2081F308BF2033A3F10B03B3F120020CDABB
S31508002B300C3208DD02F1140CC2F10C0201FA0CF099
S31508002B4021FA02F10CE002F11402D8BFC2F1200CFE
S31508002B5001FA02F120FA0CFCDCBF41EA0C019040B4
S31508002B60E41AA2BF01EB0451294330BD6FEA0404FD
S31508002B701F3C1CDA0C340EDC04F11404C4F12002E8
S31508002B8020FA04F001FA02F340EA030021FA04F3FA
S31508002B9045EA030130BDC4F10C04C4F1200220FA51
S31508002BA002F001FA04F340EA0300294630BD21FA8F
S31508002BB004F0294630BD94F0000F83F4801306BF55
S31508002BC081F480110134013D4EE77FEA645C18BF49
S31508002BD07FEA655C29D094EA050F08BF90EA020FE0
S31508002BE005D054EA000C04BF1946104630BD91EAD8
S31508002BF0030F1EBF0021002030BD5FEA545C05D1DB
S31508002C004000494128BF41F0004130BD14F5800419
S31508002C103CBF01F5801130BD01F0004545F0FE418D
S31508002C2041F470014FF0000030BD7FEA645C1ABFC2
S31508002C30194610467FEA655C1CBF0B46024650EAF9
S31508002C40013406BF52EA033591EA030F41F4002125
S31508002C5030BD00BF90F0000F04BF0021704730B5AB
S31508002C604FF4806404F132044FF000054FF0000180
S31508002C7050E700BF90F0000F04BF0021704730B541
S31508002C804FF4806404F1320410F0004548BF404216
S31508002C904FF000013EE700BF42004FEAE2014FEA6B
S31508002CA031014FEA02701FBF12F07F4393F07F4F46
S31508002CB081F06051704732F07F4208BF704793F049
S31508002CC07F4F04BF41F40021704730B54FF460745C
S31508002CD001F0004521F000411CE700BF50EA01025F
S31508002CE008BF704730B54FF000050AE050EA010208
S31508002CF008BF704730B511F0004502D5404261EB78
S31508002D0041014FF4806404F132045FEA915C3FF4B8
S31508002D10D8AE4FF003025FEADC0C18BF03325FEA55
S31508002D20DC0C18BF033202EBDC02C2F1200300FA06
S31508002D3003FC20FA02F001FA03FE40EA0E0021FA2B
S31508002D4002F11444BDE600BF70B54FF0FF0C4CF419
S31508002D50E06C1CEA11541DBF1CEA135594EA0C0FCB
S31508002D6095EA0C0F00F0DEF82C4481EA030621EA06
S31508002D704C5123EA4C5350EA013518BF52EA033541
S31508002D8041F4801143F4801338D0A0FB02CE4FF0F3
S31508002D900005E1FB02E506F00042E0FB03E54FF023
S31508002DA00006E1FB03569CF0000F18BF4EF0010E1B
S31508002DB0A4F1FF04B6F5007F64F5407404D25FEA17
S31508002DC04E0E6D4146EB060642EAC62141EA5551CA
S31508002DD04FEAC52040EA5E504FEACE2EB4F1FD0C0C
S31508002DE088BFBCF5E06F1ED8BEF1004F08BF5FEA8A
S31508002DF0500E50F1000041EB045170BD06F000463C
S31508002E0046EA010140EA020081EA0301B4EB5C04E8
S31508002E10C2BFD4EB0C0541EA045170BD41F48011E0
S31508002E204FF0000E013C00F3AB8014F1360FDEBF05
S31508002E30002001F0004170BDC4F10004203C35DAE1
S31508002E400C341BDC04F11404C4F1200500FA05F364
S31508002E5020FA04F001FA05F240EA020001F0004205
S31508002E6021F0004110EBD37021FA04F642EB06017B
S31508002E705EEA430E08BF20EAD37070BDC4F10C04A5
S31508002E80C4F1200500FA04F320FA05F001FA04F269
S31508002E9040EA020001F0004110EBD37041F1000155
S31508002EA05EEA430E08BF20EAD37070BDC4F1200560
S31508002EB000FA05F24EEA020E20FA04F301FA05F2C8
S31508002EC043EA020321FA04F001F0004121FA04F270
S31508002ED020EA020000EBD3705EEA430E08BF20EA40
S31508002EE0D37070BD94F0000F0FD101F0004640007A
S31508002EF041EB010111F4801F08BF013CF7D041EAFC
S31508002F00060195F0000F18BF704703F000465200FF
S31508002F1043EB030313F4801F08BF013DF7D043EAD0
S31508002F200603704794EA0C0F0CEA135518BF95EA86
S31508002F300C0F0CD050EA410618BF52EA4306D1D10D
S31508002F4081EA030101F000414FF0000070BD50EA2C
S31508002F50410606BF1046194652EA430619D094EAB6
S31508002F600C0F02D150EA013613D195EA0C0F05D1A0
S31508002F7052EA03361CBF104619460AD181EA0301F4
S31508002F8001F0004141F0FE4141F470014FF00000AC
S31508002F9070BD41F0FE4141F4780170BD70B54FF047
S31508002FA0FF0C4CF4E06C1CEA11541DBF1CEA1355C7
S31508002FB094EA0C0F95EA0C0F00F0A7F8A4EB0504A9
S31508002FC081EA030E52EA03354FEA013100F08880A0
S31508002FD04FEA03334FF0805545EA131343EA126369
S31508002FE04FEA022245EA111545EA10654FEA00261E
S31508002FF00EF000419D4208BF964244F1FD0404F5D7
S31508003000407402D25B084FEA3202B61A65EB030532
S315080030105B084FEA32024FF480104FF4002CB6EBEF
S31508003020020E75EB030E22BFB61A754640EA0C006F
S315080030305B084FEA3202B6EB020E75EB030E22BFAF
S31508003040B61A754640EA5C005B084FEA3202B6EBF0
S31508003050020E75EB030E22BFB61A754640EA9C00AF
S315080030605B084FEA3202B6EB020E75EB030E22BF7F
S31508003070B61A754640EADC0055EA060E18D04FEA3D
S31508003080051545EA16754FEA06164FEAC30343EADD
S3150800309052734FEAC2025FEA1C1CC0D111F4801FAA
S315080030A00BD141EA00014FF000004FF0004CB6E7A3
S315080030B011F4801F04BF01430020B4F1FD0C88BF42
S315080030C0BCF5E06F3FF6AFAEB5EB030C04BFB6EB4D
S315080030D0020C5FEA500C50F1000041EB045170BD40
S315080030E00EF0004E4EEA113114EB5C04C2BFD4EB6D
S315080030F00C0541EA045170BD41F480114FF0000EF1
S31508003100013C90E645EA060E8DE60CEA135594EA6C
S315080031100C0F08BF95EA0C0F3FF43BAF94EA0C0F6F
S315080031200AD150EA01347FF434AF95EA0C0F7FF4E4
S3150800313025AF104619462CE795EA0C0F06D152EA38
S3150800314003353FF4FDAE1046194622E750EA41061C
S3150800315018BF52EA43067FF4C5AE50EA41047FF42D
S315080031600DAF52EA43057FF4EBAE12E74FF0FF3C92
S3150800317006E000BF4FF0010C02E000BF4FF0010C63
S315080031804DF804CD4FEA410C7FEA6C5C4FEA430CDC
S3150800319018BF7FEA6C5C1BD001B050EA410C0CBF2B
S315080031A052EA430C91EA030F02BF90EA020F00208D
S315080031B0704710F1000F91EA030F58BF994208BFF4
S315080031C090422CBFD8176FEAE37040F001007047B1
S315080031D04FEA410C7FEA6C5C02D150EA013C07D108
S315080031E04FEA430C7FEA6C5CD6D152EA033CD3D053
S315080031F05DF8040B704700BF8446104662468C464D
S315080032001946634600E000BF01B5FFF7B7FF00287F
S3150800321048BF10F1000F01BD4DF808EDFFF7F4FFA8
S315080032200CBF012000205DF808FB00BF4DF808ED33
S31508003230FFF7EAFF34BF012000205DF808FB00BF56
S315080032404DF808EDFFF7E0FF94BF012000205DF878
S3150800325008FB00BF4DF808EDFFF7CEFF94BF01202D
S3150800326000205DF808FB00BF4DF808EDFFF7C4FF26
S3150800327034BF012000205DF808FB00BF4FEA410279
S31508003280B2F1E04324BFB3F5001CDCF1FE5C0DD9B6
S3150800329001F0004C4FEAC0024CEA5070B2F1004F00
S315080032A040EB830008BF20F00100704711F0804F03
S315080032B021D113F13872BCBF01F00040704741F4C8
S315080032C080114FEA5252C2F11802C2F1200C10FACC
S315080032D00CF320FA02F018BF40F001004FEAC123B0
S315080032E04FEAD32303FA0CFC40EA0C0023FA02F354
S315080032F04FEA4303CCE77FEA625307D150EA01332A
S315080033001EBF4FF0FE4040F44000704701F00040F9
S3150800331040F0FE4040F40000704700BF08B52D4B52
S31508003320D3F8945001F042F900F0010401F032FBA1
S31508003330044000F02DFC044015F0005F3CD115F068
S31508003340805F3DD101F09CF8044000F075FE044012
S3150800335000F0CEFE044001F049F9044000F0CCFC30
S31508003360044001F0C1FA044000F0C4FF044000F034
S31508003370C1F9044000F01CF9044225D106F01EFDEF
S31508003380002000F08FF9022001F004F9124B1B68A7
S315080033909B0B642202FB03F3002BF4D000BF00BF93
S315080033A000BF00BF00BF00BF00BF00BF00BF00BF17
S315080033B000BF00BF013BEFE7084801F0FFF8C1E78F
S315080033C0074801F0FBF8BDE7064B186806F069FDEB
S315080033D0FEE700BF0010024094000020010000092B
S315080033E0020000093401002008B5054A00210548F5
S315080033F006F0F9FC044B1860003818BF012008BD18
S315080034003CCC00081D3300083401002000B585B007
S31508003410EC468CE80F0000231A466146054800680A
S3150800342006F05DFF0121044B186806F0E7FD05B0BC
S315080034305DF804FB440100204001002008B5014660
S31508003440024B186806F0DAFD08BD00BF40010020EF
S3150800345030B589B08BE000231A4602A94E480068A9
S3150800346006F07FFF9DF808509DF81130012B12D009
S31508003470022B35D0002B40F08780082D3CD86AB245
S31508003480002A69D0013D072D66D8DFE805F03D41E1
S3150800349045654C4F5B62142D0DD9404801F08EF8F6
S315080034A0FF238DF818309DF81130059A012106A8DA
S315080034B000F06EFF68E0284600F036FB01908DF8B4
S315080034C0185004220DF119010DEB020001F078FFE6
S315080034D09DF81130059A052106A800F059FF53E01A
S315080034E004220DEB02010DF1090001F069FF0199B3
S315080034F0284600F0A9FA47E0FF2D2DD1002000F05C
S31508003500D1F803F005FA3FE0012000F0CBF83BE0E4
S31508003510002000F0C7F837E040F6B831204B1868AD
S3150800352006F030FD30E001F043F82DE006228DF874
S3150800353018200A228DF81920059A022106A800F0FB
S3150800354027FF21E000F036FBF0B9164801F036F8FF
S315080035501AE000F04FFB17E0134801F02FF813E0CC
S31508003560022001F017F812E0002000F09BF84FF057
S31508003570FF33002207210D48006806F08CFD04463B
S3150800358010F0010F7FF467AF14F0020FE8D114F0C2
S31508003590040FECD0E8E700BF440100200100000852
S315080035A0380100200400000802000008400100203D
S315080035B070B52A4806F000FD294B1860041E18BF8E
S315080035C00124284A0021284806F00DFC274B1860DC
S315080035D000280CBF002404F00104254A1021082005
S315080035E006F032FE234B186000280CBF002404F0B6
S315080035F00104214D214B02220121284606F06EFCCA
S315080036001F4E306000280CBF002404F001041D4B37
S3150800361004220121284606F061FC1B4D286000287B
S315080036200CBF002404F001044FF47A71306806F0E8
S31508003630A9FC002814BF002404F0010440F6B831A0
S31508003640286806F09FFC002814BF002404F0010433
S315080036500E4800F0C5FE204670BD00BFD8CC000855
S315080036604001002000CD0008513400084801002020
S31508003670E8CC0008440100203D340008C8CC000806
S315080036803C010020B8CC0008380100200D340008A1
S3150800369008B50146024B186806F0B0FC08BD00BF25
S315080036A04C01002010B504460146032000F036FF01
S315080036B02146122000F02AFA10BD08B5122000F0A3
S315080036C047FA08BD08B5F2EE087AB4EEE70AF1EE55
S315080036D010FA01DDB0EE670AF9EE047AB4EEE70AED
S315080036E0F1EE10FA01D5B0EE670A00F049FD00F0D8
S315080036F0010008BD38B5174A0021174806F073FBC4
S31508003700164B1860041E18BF0124154806F054FC11
S31508003710144B186000280CBF002404F00104124B57
S3150800372001221146114806F0D9FB114D28600028E0
S315080037300CBF002404F001049FED0E0AFFF7C2FF38
S31508003740C821286806F01EFC002814BF002004F0D3
S31508003750010038BD78CD00087937000854010020EB
S3150800376058CD00084C01002068CD000891360008A5
S31508003770500100200000000008B52DED0C8BDFED90
S31508003780759AB0EE699AF0EE698AB0EE698A45E0F4
S315080037900020FFF787FF704800F010FF6FE09FEDED
S315080037A06D9AF4EEE7CAF1EE10FA02D57CEEE76AF6
S315080037B001E0DFED686AB4EEC79AF1EE10FA07D4B5
S315080037C0F4EEC76AF1EE10FA00F39580B0EE479A68
S315080037D03DEE0D7A78EEEAAA27EE2A7ADFED5F6AE1
S315080037E06BEEA66A37EE267AF1EE479A79EE277AD5
S315080037F077EEC77AF4EECC7AF1EE10FA06DCF4EE40
S31508003800EC7AF1EE10FA79D4B0EE67CAB0EE4C0A4B
S31508003810FFF758FF10B9524800F0D0FEF0EE69BA2B
S31508003820B0EE49BAF0EE68AAB0EE48AA4FF0FF33F8
S31508003830002201214B48006806F02DFC10F0010F0C
S31508003840F4D0494803F053FFFFF737FF9FED418A4D
S31508003850F0EE488AB0EE489AF0EE489A0028DDD095
S31508003860002000F075F900284BD10E2000F074F9FD
S31508003870DFED3E7AB4EEE70AF1EE10FA88DC0220B4
S3150800388000F06AF9B0EE409A032000F065F9F0EE10
S31508003890409A042000F060F9B0EE40DA062000F005
S315080038A05BF9B0EE40CA072000F056F9F0EE40CAC0
S315080038B0092000F051F9F0EE408A052000F04CF995
S315080038C038EEC08A69EE087AB6EE007A29EE877A6B
S315080038D0DFED276A27EE267A3AEE08AA27EE0A7A55
S315080038E037EE0B7AB4EEE7CAF1EE10FA7FF757AF68
S315080038F03CEE679A55E7B0EE669A69E7B0EE6CCA91
S3150800390084E7002000F024F9012808D0F0EE6B9A2D
S31508003910B0EE4B9AF0EE6A8AB0EE4A8A7EE700F07D
S315080039201BF9FFF7CFFE40B1DFED0A9AB0EE699AB0
S31508003930F0EE698AB0EE698A70E70E4800F03EFE3E
S31508003940DFED049AB0EE699AF0EE698AB0EE698AFC
S3150800395064E700BF00000000040000079A99193FB9
S31508003960020000074C010020640300200000DC422E
S31508003970CDCC4C3E0100000701288CBF0020012059
S3150800398070470000084B03EB00139B688B4207D86F
S31508003990054B03EB0013DB688B4203D2002070470C
S315080039A00020704701207047B8CD0008084B03EB8C
S315080039B000139B688B4207DC054B03EB0013DB689F
S315080039C08B4203DA002070470020704701207047B9
S315080039D0B8CD00080C4B03EB0013D3ED027AF4EED6
S315080039E0C07AF1EE10FA0BD8074B03EB0013D3EDB0
S315080039F0037AF4EEC07AF1EE10FA03DA0020704783
S31508003A000020704701207047B8CD000808B50301AB
S31508003A100C4AD35C13F0010F09D113F0020F0BD136
S31508003A2013F0040F0BD00846FFF7A6FF03E000EEDD
S31508003A30101AFFF7CFFF08BDFFF7B8FFFBE7FFF740
S31508003A40A1FFF8E7B8CD000838B504460301144AC3
S31508003A50D35C13F0080F13D10D464FF0FF31114B0D
S31508003A60186806F09BFB29462046FFF7CFFF78B17A
S31508003A700D4B43F834500B4B186806F0BEFB38BDA7
S31508003A80000240F0C06040F0040000F097FDF6E741
S31508003A90200240F0C06040F0080000F08FFDEAE721
S31508003AA0B8CD0008580100205C01002038B504464E
S31508003AB00D464FF0FF31134B186806F06FFB082CC4
S31508003AC00CD029462046FFF7A1FF60B10E4B43F8FC
S31508003AD034500C4B186806F090FB38BD00F052FCC9
S31508003AE00828F3D1EDE7084B03EBC4031A7942F033
S31508003AF002021A71200240F0C06040F0100000F087
S31508003B005DFDE3E7580100205C01002008B5FFF7DA
S31508003B10CDFF08BD00B583B08DED010A0199FFF709
S31508003B20C5FF03B05DF804FB38B50446064D4FF0F3
S31508003B30FF31286806F032FB044B53F834402868F6
S31508003B4006F05BFB204638BD580100205C010020CA
S31508003B5008B5FFF7E9FF08BD08B5FFF7E5FF00EE72
S31508003B60100A08BD08B5034B03EB00135968FFF7A5
S31508003B709DFF08BDB8CD000810B5002404E0E0B2EA
S31508003B80FFF7F0FF0134A4B2142CF8D910BD0000D9
S31508003B9010B5064806F0B9FA054B1860041E18BF9A
S31508003BA00124FFF7E9FF204610BD00BFA8CD000895
S31508003BB05801002038B500F0DDFE00F001050024AC
S31508003BC001E00134E4B2142C0ED82301084AD35C70
S31508003BD013F0100FF5D02046FFF7A6FF0146204642
S31508003BE000F09BFE0540ECE700F0B6FE284038BD25
S31508003BF0B8CD000830B583B00024012501E00134B2
S31508003C00E4B2142C10D82301124AD35C13F0100F17
S31508003C10F5D001A9204600F079FE0540EFD00199BC
S31508003C202046FFF743FFEAE70DB103B030BD0A4867
S31508003C3000F0C4FC002401E00134E4B2142CF4D8EA
S31508003C402301044AD35C13F0100FF5D02046FFF782
S31508003C5089FFF1E7B8CD00082000000608B572B163
S31508003C600D4B60F07F00187000225A7099700B484F
S31508003C700323838100F0C8FC00F0010008BD064B51
S31508003C8060F07F001870597004480223838100F0A1
S31508003C90BBFC00F00100F1E708020020000000204C
S31508003CA010B50C4692B1114B187000225A709A70D2
S31508003CB00F480323838100F0A7FC00F001000D4B99
S31508003CC05A789B7843EA0223238010BD074B187065
S31508003CD000225A7006480223838100F095FC00F002
S31508003CE00100044B5B782380EFE700BF0802002041
S31508003CF0000000201002002038B5144806F005FA26
S31508003D00134D2860041E18BF01244FF0FF3106F03A
S31508003D1045FA002000F094FB002282211046FFF7A6
S31508003D209DFF0440002000F09BFB012000F088FB6B
S31508003D30002282211046FFF791FF0440012000F07F
S31508003D408FFB286806F059FA204638BD14CF0008BC
S31508003D50040200202DE9F04182B00F469046002368
S31508003D600B70ADF8063018B1012854D0012600E0D2
S31508003D700126404D4FF0FF31286806F00FFA30460D
S31508003D8000F05EFB0022A0211046FFF767FF00F057
S31508003D900104304600F064FB286806F02EFA642019
S31508003DA006F08EF84FF0FF31286806F0F7F930462E
S31508003DB000F046FB01220DF106011046FFF770FFE1
S31508003DC00440304600F04CFB286806F016FA24B387
S31508003DD0BDF8063013F0010F24D15B08ADF80630A4
S31508003DE0A8F80030234D4FF0FF31286806F0D6F9C1
S31508003DF0304600F025FB002284211046FFF72EFFEF
S31508003E000440304600F02CFB286806F0F6F92046F8
S31508003E1002B0BDE8F0810026ABE73B7843F0020329
S31508003E203B70F4E7134C4FF0FF31206806F0B6F903
S31508003E30304600F005FB002239460720FFF730FF21
S31508003E40304600F00DFB304600F0FAFA00228221D7
S31508003E501046FFF703FF304600F002FB206806F025
S31508003E60CCF93B7803F0FC033B7043F001033B704D
S31508003E700024CCE704020020F0B585B0012006F046
S31508003E801FF808226249634802F01AF89EE00424E3
S31508003E904FF0FF31604B186806F080F900230AE0FE
S31508003EA0E1185B4A32F8111004AA02EB830242F8C1
S31508003EB0101C01339BB2032BF2D91420FFF74CFEDA
S31508003EC0002325E004AA02EB830252ED047AF8EEF9
S31508003ED0677A9FED527A67EE877A9FED517A67EE99
S31508003EE0877A67EE807A4F4A02EB830292ED007A70
S31508003EF067EE277A4C4A02EB830292ED007A77EE58
S31508003F00C77A4A4A02EB8302C2ED007A01339BB2B2
S31508003F10032BD7D9002401E00134A4B2032C1DD801
S31508003F20424B03EB84031868FEF7B6FE06460F46B7
S31508003F3033A3D3E90023FFF78DF90028ECD032A389
S31508003F40D3E9002330463946FFF770F90028E3D055
S31508003F50364B03EB840300221A60DDE7334C94EDFD
S31508003F60020A0B20FFF7D6FD94ED030A0C20FFF793
S31508003F70D1FDD4ED037AF5EE407AF1EE10FA36D19A
S31508003F809FED2B0A0D20FFF7C5FD284C94ED020A7C
S31508003F90D4ED037A20EE270A0E20FFF7BBFD94ED39
S31508003FA0000A0F20FFF7B6FD94ED010A1020FFF76F
S31508003FB0B1FD94ED000AD4ED017A20EE270A11200E
S31508003FC0FFF7A8FD144B186806F017F94FF0FF33F2
S31508003FD0002203211748006806F05DF810F0020F6A
S31508003FE07FF455AF10F0010FF0D0002450E70F4BC7
S31508003FF093ED020A80EE270A0D20FFF78BFDC4E732
S315080040009A9999999999A9BF9A9999999999A93F24
S315080040103402002070040020280200200000803DA1
S3150800402000008039A4CF000894CF000818020020A9
S31508004030000000002C02002010B50F4A00210F488E
S3150800404005F0D1FE0E4B1860041E18BF01240D485A
S3150800405005F0B2FF0C4B186000280CBF002404F0D2
S3150800406001040A4806F051F8094B186000280CBFED
S31508004070002004F0010010BD70CF0008793E00084A
S315080040803002002060CF00082C02002050CF000824
S315080040902802002008B50221024B186805F0AEFF79
S315080040A008BD00BF2C02002008B50121024B186884
S315080040B005F0A4FF08BD00BF2C02002008B5836DDB
S315080040C033B9C36CD86B40F0806000F077FA08BD4E
S315080040D0806D40F0407000F071FAF8E708B50146C7
S315080040E0024B186805F08AFF08BD00BF4C02002085
S315080040F038B51A4A00211A4805F075FE194B18609A
S31508004100041E18BF0124184805F056FF174B1860FF
S3150800411000280CBF002404F00104154B01221146A7
S31508004120144805F0DBFE144D286000280CBF002457
S3150800413004F001040021114802F08BFC002814BF8A
S31508004140002404F001043221286805F01BFF00282A
S3150800415014BF002004F0010038BD00BF08D00008D5
S31508004160CD42000854020020E8CF00084C02002087
S31508004170F8CF0008DD40000850020020C8030020E0
S3150800418008B5064B83ED000A0121054B186805F0B2
S3150800419035FFB0FA80F0400908BD00BF4402002090
S315080041A04C0200200000000008B52DED028B10EE31
S315080041B0100AFEF771FD11A3D3E90023FEF70EFCE2
S315080041C010A3D3E90023FEF7E9FEFFF757F808EE38
S315080041D0100ADFED097A28EE278A1420FFF7BCFCBF
S315080041E0C8EE007AFCEEE77A17EE900ABDEC028B71
S315080041F008BD00BFAFF3008000F07F454A0C022BD4
S3150800420087163440166BB8C83D0D414000000000C3
S3150800421008B52DED028B2A4BD3ED007A294B93ED89
S31508004220008AF4EEC87AF1EE10FA26D517EE900A4F
S31508004230FEF732FD20A3D3E90023FEF7CFFBFFF7F5
S315080042401DF807EE900A1E4B1860B4EEE78AF1EEE9
S3150800425010FA01D583ED008A194B93ED000AFFF792
S31508004260A3FF034600221146174802F024FCB0FAC1
S3150800427080F04009BDEC028B08BDF4EEC87AF1EE79
S3150800428010FAE9DD17EE900AFEF706FD0AA3D3E950
S315080042900023FEF7A1FBFEF7F1FF07EE900A084B95
S315080042A01860B4EEE78AF1EE10FAD5DD83ED008AE0
S315080042B0D2E700BFAFF300809A9999999999B93FC7
S315080042C04802002044020020C803002008B54FF029
S315080042D0FF33002201210648006805F0DCFE10F0D5
S315080042E0010FF4D0FFF794FF002000F033F9EEE752
S315080042F04C02002070B5042000F02CF91D4C2378E0
S3150800430003432370032000F025F9237843EA40038A
S315080043102370022000F01EF9237843EA80032370F5
S31508004320012000F017F9237843EAC000C0B22070D4
S31508004330114E336843EA40133360104D104928463E
S3150800434001F05FFF04463146284601F05AFF044350
S31508004350E4B2284601F0D8FF0443E4B20221284615
S3150800436002F01AF9204310F0FF0F0CBF01200020BD
S3150800437070BD00BF58020020440000200004002041
S315080043806C000020014B1878704700BF58020020C7
S31508004390082901D90020704700B587B012021FFA14
S315080043A082FC4CEA03130C4A1278134343F4107345
S315080043B00093002301930293039304918DF814301C
S315080043C0012302466946054801F0CCFFB0FA80F0A1
S315080043D0400907B05DF804FB5802002000040020DD
S315080043E0014B1860704700BF5C02002030B58FB0E3
S315080043F005AB07AA002102F02AF8079BC3F300229F
S315080044000492C3F301138DF80D309DF82C208DF816
S315080044100C2001AC214605A800F0D2FF034B1D680D
S3150800442094E80F00A8470FB030BD00BF5C0200201B
S3150800443008B5406A40F0807000F0C0F808BD00007A
S3150800444008B5064B4FEA401C03EB4010027F8188F3
S3150800445053F80C0003F051F808BD00BF2CD0000833
S3150800446008B5064B4FEA401C03EB4010027E8188D4
S3150800447053F80C0003F041F808BD00BF2CD0000823
S3150800448070B582B0224B1A6E42F001021A661B6E94
S3150800449003F001030193019B012500240BE000238F
S315080044A01D401C4B4A0103EB41110431985802F098
S315080044B045FF0134E4B2042C08D82146154B03EB1A
S315080044C044139B68002BEAD10123E9E700240EE098
S315080044D001231D402046FFF7C3FF0F4B720103EB74
S315080044E046110431985802F029FF0134E4B2032C2E
S315080044F00AD82646084B03EB44139B68012BE8D0E1
S31508004500112BE5D00023E4E7284602B070BD00BFB2
S3150800451000100240ACD000082CD0000808B559B1EC
S315080045200B4B4FEA401C03EB4010027F818853F87F
S315080045300C0002F0E2FF08BD054B4FEA401C03EBF6
S315080045404010027E818853F80C0002F0D6FFF2E78D
S315080045502CD0000838B504460D4B420103EB401534
S31508004560A988985802F0C2FFEB69012B07D0084BBF
S3150800457003EB44139B69012B05D0002038BD0128A5
S31508004580F5D10120FAE708B10020F7E70120F5E7A1
S31508004590ACD0000808B5044B420103EB40108188F3
S315080045A0985802F0AFFF08BD2CD0000801207047CC
S315080045B008B500211320FFF7A9FA08BD08B501467A
S315080045C01320FFF7A3FA08BD0246002008B1002011
S315080045D0704700EB8003044951F823309342F7D023
S315080045E0431CD8B2F2E700BF4CD1000808B504480E
S315080045F005F0E2FC034B1860003818BF012008BD1F
S3150800460084D100086002002038B504460378244D9A
S3150800461003EB830305EB83034FF0FF31586805F07E
S31508004620BDFD237803EB830305EB8303D96841F0CB
S3150800463002011C4B186805F00EFD237803EB830076
S31508004640A389A268616855F8200004F02BF90028B0
S315080046500CBF0125002511D00020237810F0020F89
S3150800466005F0010518BF002503EB83030C4A02EB8E
S315080046708303586805F0C1FD284638BD237803EB47
S315080046808303074A02EB8303D9684FF0FF330022FE
S3150800469041F002010348006805F0FDFCDDE700BFB4
S315080046A04CD100086002002008B5FFF78DFF00EB2B
S315080046B08000044B03EB8003D968034B186805F0A8
S315080046C09DFC08BD4CD100086002002008B5FFF724
S315080046D07BFF00EB8000044B03EB8003D968034B98
S315080046E0186805F08BFC08BD4CD100086002002054
S315080046F010B50446006E40F00070FFF75FFF2046D5
S31508004700FFF762FF0221024B186805F077FC10BD1F
S315080047106002002007EE900AF8EEE77A9FED097A24
S3150800472087EE870ADFED087A60EE277A9FED077A2B
S3150800473077EE877A20EE270ADFED057A30EE670AEC
S31508004740704700BFECB9FE45DB8A1F416DE76B4336
S3150800475042E0754310B584B000238DF80F300A2067
S3150800476005F0AEFB01248FE09DF80F0010F0010F55
S315080047702CD010F0800F05D110F0400F05D0544B07
S3150800478001932BE0534B019328E010F0200F08D03B
S315080047904F4B019340F0A46040F48020FFF70EFFD2
S315080047A01CE010F0100F02D0494B0193F2E710F00D
S315080047B0080F02D0464B0193ECE710F0040F02D025
S315080047C0434B0193E6E7424B0193E3E710F0020FF0
S315080047D009D03F4B01934048FFF7F0FE00238DF8C0
S315080047E00F3001245FE03A4B01933C48FFF7E6FEA1
S315080047F0F4E79DF80F0010F0010F2CD010F0800F91
S3150800480005D110F0400F05D0314B02932BE0314B08
S31508004810029328E010F0200F08D02D4B029340F0A9
S31508004820A26040F48020FFF7C9FE1CE010F0100FCC
S3150800483002D0274B0293F2E710F0080F02D0244B60
S315080048400293ECE710F0040F02D0214B0293E6E73F
S315080048501F4B0293E3E710F0020F33D01C4B029371
S315080048601F48FFF7ABFE00238DF80F3001249DED9E
S31508004870010A0820FFF74EF99DED020A0920FFF705
S3150800488049F9642005F01CFB03AA0DF10F0100206D
S31508004890FFF760FA04403FF467AFBDF80C00FFF776
S315080048A039FF8DED010A03AA0DF10F010120FFF76B
S315080048B051FA04409DD0BDF80C00FFF72BFF8DED93
S315080048C0020AD4E7024B02930648FFF777FECAE7C7
S315080048D07B9488C30040834500002105000022051B
S315080048E0000011050000120508B5054A0021054813
S315080048F005F079FA044B1860003818BF012008BD86
S31508004900B0D10008554700086402002008B504F035
S315080049101BFDB0FA80F0400908BD70B505460E4685
S3150800492005F0D6F9044610F4807F04D10120E4B2DC
S31508004930FF2C0ED070BD04F025FB0443A4B231460B
S31508004940284605F0C5F9204380B2B0FA80F0400940
S31508004950EDE70020EEE7000010B502F08BFBB0FA99
S3150800496080F46409024B186805F047FC204610BD20
S315080049706802002008B54FF0FF31054B186805F0AE
S315080049800DFC02F05FFBB0FA80F0400908BD00BFDD
S315080049906802002010B50B4805F0B7FB0A4B1860F3
S315080049A0041E18BF0124FFF7E5FF0440002004F0A9
S315080049B085FE002814BF002404F00104FFF7CCFF8D
S315080049C0204010BDE0D1000868020020014A024BD1
S315080049D09A6070470028000800ED00E02DE9F041D4
S315080049E088B0002403940494059406940794364BDF
S315080049F0DA6C42F00402DA64DA6C02F0040200921D
S31508004A00009ADA6C42F00102DA64DA6C02F001020A
S31508004A100192019ADA6C42F00202DA64DB6C03F066
S31508004A2002030293029B294F22464FF480413846DF
S31508004A3002F063FD22464FF480714FF0904002F079
S31508004A405CFD234D22466021284602F056FD4FF4B0
S31508004A5080430393012604960594069403A93846D1
S31508004A6002F06CFC4FF40048CDF80C8004940594D1
S31508004A7003A9384602F062FC4FF480730393049648
S31508004A800594069403A94FF0904002F057FCCDF820
S31508004A900C800494059403A94FF0904002F04EFC54
S31508004AA0982303930494059403A9284602F046FC28
S31508004AB06023039304960594069403A9284602F0F6
S31508004AC03DFC08B0BDE8F08100100240000800482F
S31508004AD00004004800B583B0164B9A6C42F00102F8
S31508004AE09A649A6C02F001020092009A9A6C42F05B
S31508004AF002029A649B6C03F002030193019B002255
S31508004B0005210C2001F0F0FE0C2001F0FDFE00222C
S31508004B1005210D2001F0E8FE0D2001F0F5FE00222A
S31508004B2005213A2001F0E0FE3A2001F0EDFE03B03F
S31508004B305DF804FB0010024008B5FEF755FC024B71
S31508004B40186805F0AEF9FEE76C02002008B50020EB
S31508004B50FEF7A8FD01F0DCFE72B6FEE700B587B0E9
S31508004B6000230093019302930393049305932F481C
S31508004B702F4A026043608360C360012202610821F4
S31508004B804161037642760421C16180F82030836250
S31508004B90C36280F83020436380F838201C21C16343
S31508004BA0802101644364826400F09EFC002832D1AF
S31508004BB0204B009306230193072302937F23039335
S31508004BC004230493002305936946184800F0ECFE75
S31508004BD018BB194B00930C2301936946134800F040
S31508004BE0E3FEE0B9154B00931223019369460F487B
S31508004BF000F0DAFEA8B9124B009318230193694610
S31508004C000A4800F0D1FE70B97F21084801F002FA7F
S31508004C1007B05DF804FBFFF799FFFFF797FFFFF76B
S31508004C2095FFFFF793FFFFF791FF00BF7004002081
S31508004C300000045040002019000021438000501D48
S31508004C400080F03E08B50D480D4B036020234360F5
S31508004C5000238360C3604FF4402202614FF4A00230
S31508004C6042610376437683760122C27603774377D9
S31508004C7001F021FA00B908BDFFF768FF000400201B
S31508004C800064004000B58BB02422002101A807F07B
S31508004C90DAFE1048104B036001F0C9FE98B90022ED
S31508004CA00192029203920492059201A9094801F021
S31508004CB019FF50B9002201A9064801F0AEFF30B924
S31508004CC00BB05DF804FBFFF741FFFFF73FFFFFF767
S31508004CD03DFF00BFC80300200074004008B5104817
S31508004CE0104B03604FF482734360002383604FF4D4
S31508004CF0E062C2600361012242614FF40072826180
S31508004D003022C2610362436283620722C26203637E
S31508004D10436303F057FD00B908BDFFF717FF00BF4F
S31508004D20000300200030014008B51148114B03600C
S31508004D30114B4360002383600122C2600361436113
S31508004D408361C361036202F0E6FB50B9002108489B
S31508004D5002F03FFC38B90021054802F068FC20B98A
S31508004D6008BDFFF7F3FEFFF7F1FEFFF7EFFE00BF02
S31508004D707403002000540040EC9C901008B50848C5
S31508004D80084B03600623436040F6FF73C36096230F
S31508004D90836002F078FC00B908BDFFF7D7FE00BFB4
S31508004DA0640300200030004008B50848084B03603B
S31508004DB0002303714371436183610123036201F098
S31508004DC0BFFD00B908BDFFF7C1FE00BFDC03002028
S31508004DD00030024000B597B04422002105A807F02C
S31508004DE032FE0023009301930293039304934FF436
S31508004DF0007002F08BFC30BB092305934FF4A02307
S31508004E00069301230A9302230F9303221092042286
S31508004E10119210221292072213921493159305A841
S31508004E2002F05EFD88B90F23009303230193002344
S31508004E300293039304930421684603F087F830B974
S31508004E4017B05DF804FBFFF781FEFFF77FFEFFF75B
S31508004E507DFE000008B5FFF7B9FD00F0E1FAFFF79F
S31508004E60B9FFFFF7BBFDFFF735FEFFF777FEFFF744
S31508004E70E9FEFFF707FFFFF731FFFFF755FFFFF7DB
S31508004E807DFFFFF791FF04F06BFF054A00210548F7
S31508004E9004F0A9FF044B186004F074FFFEE700BF96
S31508004EA0F8D10008394B00086C02002000B583B021
S31508004EB00D4B1A6E42F001021A661A6E02F00102D2
S31508004EC00092009A9A6D42F080529A659B6D03F0A3
S31508004ED080530193019B00220F216FF0010001F01E
S31508004EE003FD03B05DF804FB0010024070B59EB0E8
S31508004EF00446002119911A911B911C911D91542267
S31508004F0004A807F0A0FD2268334B9A4201D01EB0D0
S31508004F1070BD4FF4804304934FF04053169304A892
S31508004F2003F08EF9002850D12C4BDA6C42F400526B
S31508004F30DA64DA6C02F400520192019ADA6C42F0F1
S31508004F400102DA64DA6C02F001020292029ADA6C61
S31508004F5042F00202DA64DB6C03F002030393039B5C
S31508004F60062319930B261A9600251B9519A94FF0A7
S31508004F70904002F0E3F9032319931A961B9519A991
S31508004F80174802F0DBF91748174B03604560856040
S31508004F90C560802303614FF4807343614FF48063D7
S31508004FA083612023C3614FF40053036201F0DAFEE4
S31508004FB070B90C4BE3649C6200220521122001F0B3
S31508004FC093FC122001F0A0FCA1E7FFF7BFFDABE7B9
S31508004FD0FFF7BCFDEDE700BF0000045000100240DB
S31508004FE000040048280400203004024000B589B0B7
S31508004FF00023039304930593069307930268244BAF
S315080050009A4202D009B05DF804FB03F5D6339A6DCF
S3150800501042F000729A659A6D02F000720192019A46
S31508005020DA6C42F00102DA64DB6C03F001030293E6
S31508005030029B4FF4C053039302230493032306935E
S315080050400923079303A94FF0904002F077F900224D
S315080050500521132001F048FC132001F055FC00221D
S315080050600521142001F040FC142001F04DFC00221B
S315080050700521152001F038FC152001F045FC002219
S315080050800521162001F030FC162001F03DFCB9E799
S31508005090006400400268094B9A4200D0704782B00B
S315080050A0A3F500539A6C42F480529A649B6C03F4FD
S315080050B080530193019B02B0704700BF0030024045
S315080050C000B589B0002303930493059306930793C9
S315080050D00268124B9A4202D009B05DF804FB03F548
S315080050E0CE339A6D42F000529A659A6D02F00052DC
S315080050F00192019ADA6C42F00102DA64DB6C03F081
S3150800510001030293029B102303930323049303A929
S315080051104FF0904002F012F9DEE700BF007400403D
S3150800512010B59CB0044600211791189119911A914F
S315080051301B91542202A807F086FC2268184B9A4253
S3150800514001D01CB010BD4023029302A803F078F8E2
S3150800515018BB144CE36C43F00103E364E36C03F0FF
S3150800516001030093009B4FF4C0631793122318930F
S315080051700023199303231A9304231B9317A94FF0AB
S31508005180904002F0DBF8A36D43F40013A365A36D0A
S3150800519003F400130193019BD3E7FFF7D7FCD8E785
S315080051A0005400400010024010B588B00023039355
S315080051B0049305930693079302682F4B9A4201D0EE
S315080051C008B010BD044603F560431A6E42F48052D7
S315080051D01A661A6E02F480520192019ADA6C42F04B
S315080051E00102DA64DB6C03F001030293029BE023FD
S315080051F0039302230493032306930523079303A922
S315080052004FF0904002F09AF81C481D4B03600123AA
S31508005210436000238360C360802202614361836127
S31508005220C361036201F09EFD00BB144BA3659C623B
S315080052301448154B03600123436010238360002341
S31508005240C3608022026143618361C361036201F026
S3150800525089FD70B90B4B63659C62002205212320EA
S3150800526001F042FB232001F04FFBA9E7FFF76EFC94
S31508005270DBE7FFF76BFCEDE700300140B8020020E2
S315080052801C000240700200203000024008B50020D1
S31508005290FEF708FA01F03CFBFEE708B50020FEF72A
S315080052A001FA01F035FBFEE708B50020FEF7FAF92A
S315080052B001F02EFBFEE708B50020FEF7F3F901F032
S315080052C027FBFEE708B50020FEF7ECF901F020FB06
S315080052D0FEE7704708B500F0B3F806F0DDFC0128D4
S315080052E000D108BD07F07EF9FBE7000008B50248C3
S315080052F001F01FFE08BD00BFB802002008B502482D
S3150800530001F017FE08BD00BF7002002008B502486C
S3150800531000F0DEF908BD00BF7004002008B5024899
S3150800532001F057F908BD00BF0004002008B502487F
S3150800533001F04FF908BD00BF0004002008B5024877
S3150800534001F047F908BD00BF0004002008B502486F
S3150800535001F03FF908BD00BF0004002008B5024867
S3150800536003F02EFC08BD00BF0003002008B5024864
S3150800537001F0DFFD08BD00BF280400200E4AD2F860
S31508005380883043F47003C2F888300C4B1A6842F030
S3150800539001021A60002199601A6822F0A85222F4C4
S315080053A010221A604FF48052DA601A6822F48022BA
S315080053B01A609961704700BF00ED00E000100240D6
S315080053C008B50B460146184607F0C2FB08BD0000A3
S315080053D0104B1B780BB90120704710B504464FF4E3
S315080053E07A70B0FBF3F30C4A1068B0FBF3F001F0E7
S315080053F093FA68B90F2C01D901200AE00022214648
S315080054004FF0FF3001F070FA044B1C60002000E0FA
S31508005410012010BD98000020940000209C00002068
S3150800542010B5032001F04EFA0F20FFF7D1FF10B197
S315080054300124204610BD0446FFF738FDF9E70000B1
S31508005440034B1B78034A11680B441360704700BF6F
S3150800545098000020D4040020014B1868704700BF4C
S31508005460D404002038B50446FFF7F6FF0546B4F124
S31508005470FF3F02D0044B1B781C44FFF7EDFF401B8F
S31508005480A042FAD338BD00BF9800002010B43030CF
S315080054900B0A9B0003F00C03C45801F01F014FF0E0
S315080054A01F0C0CFA01FC24EA0C0CC2F384628A4035
S315080054B04CEA0202C2505DF8044B704710B414302F
S315080054C04B0E9B0003F00403C458C1F304514FF07C
S315080054D0070C0CFA01FC24EA0C0C8A404CEA02027E
S315080054E0C2505DF8044B704730B583B00023019372
S315080054F0002800F0DA800446436D13B323689A68DF
S3150800550012F0005F05D09A6822F0204222F03F028E
S315080055109A602268936813F0805F1FD1936823F01E
S31508005520104323F03F0343F080539360604B1B689E
S315080055309B09604AA2FB03239B0901335B00019385
S3150800554009E0FFF7D3FC0023A36584F85030D5E7BC
S31508005550019B013B0193019B002BF9D122689368BB
S3150800556013F0805F78D1636D43F010036365A36D14
S3150800557043F00103A3650120936813F0040300D0E8
S315080055800123616D11F0100F40F08880002B40F068
S315080055908580636D23F4817343F002036365936822
S315080055A013F0010F0BD1444B9B6813F0010F06D182
S315080055B0636842498A6822F47C1213438B60627ED0
S315080055C0636B43EA4233E2681343A268134394F8D1
S315080055D0202043EA0243012A40D0A26A22B102F4FB
S315080055E07072E16A0A4313432168CD68344A2A4037
S315080055F01A43CA6021688B6813F0040300D001239C
S315080056008A6812F0080200D00122B3B9AAB9237E2B
S3150800561094F83020520042EA8332CB6823F4804360
S3150800562023F002031343CB6094F83830012B1AD0C9
S315080056302268136923F0010313612369012B24D01F
S315080056402268136B23F00F031363636D23F00303C0
S3150800565043F00103636526E000208DE7626A013A9C
S3150800566043EA4243B9E721680B6923F4FF6323F051
S315080056700403E26B256C2A43656C2A43A56C2A430E
S31508005680134343F001030B61D7E721680B6B23F043
S315080056900F03E269013A13430B63D6E7636D43F0E0
S315080056A010036365012003B030BD0120FBE700BF8E
S315080056B094000020632D3E050000045000030450AA
S315080056C007C0F0FF08B5806AFEF7EEFC08BD704714
S315080056D070B5044603681E685D6816F0020F10D0A0
S315080056E015F0020F0DD0436D13F0100F03D1436D63
S315080056F043F400634365204600F0DCFC236802227D
S315080057001A6016F0040F02D015F0040F05D116F032
S31508005710080F3AD015F0080F37D0636D13F0100F45
S3150800572003D1636D43F4007363652368DA6812F482
S31508005730406F24D1DA6812F4005F20D11A6812F09B
S31508005740080F1CD09A6812F0040F10D15A6822F07C
S315080057500C025A60636D23F480736365636D13F4FA
S31508005760805F0CD1636D43F00103636507E0636DE9
S3150800577043F010036365A36D43F00103A365204658
S31508005780FEF788FC23680C221A6016F0200F02D058
S3150800579015F0200F05D116F0400F4CD015F0400F2C
S315080057A049D0636D13F0100F03D1636D43F40053B2
S315080057B063652368DA6C12F0C00F2AD10121DA6812
S315080057C012F4406F27D10120DA6871B312F0007F16
S315080057D003D050B312F4005F27D1196811F0400FB7
S315080057E023D012F4001F20D19A6812F0080F14D1A2
S315080057F05A6822F060025A60636D23F48053636529
S31508005800636D13F4807F10D1636D43F00103636504
S315080058100BE00021D3E70020D6E7636D43F01003C1
S315080058206365A36D43F00103A365204600F03EFCC3
S31508005830236860221A6016F0800F02D015F0800FD8
S315080058402DD116F4807F02D015F4807F32D116F45C
S31508005850007F02D015F4007F38D116F0100F17D04C
S3150800586015F0100F14D0636B23B12368DB6813F0AF
S31508005870010F0AD0636D43F480636365A36D43F03B
S315080058800203A3652046FEF719FC236810221A6056
S3150800589016F4806F02D015F4806F23D170BD636D46
S315080058A043F4803363652046FFF711FF236880229F
S315080058B01A60C6E7636D43F400336365204600F05B
S315080058C0F7FB23684FF480721A60C0E7636D43F4F0
S315080058D080236365204600F0ECFB23684FF40072D2
S315080058E01A60BAE7636D43F480436365A36D43F0BA
S315080058F00803A36523684FF480621A60204600F007
S31508005900D6FBCBE708B50346806A426D12F0500F06
S3150800591030D1436D43F40073436503681A6812F087
S31508005920080F14D0DA6812F4406F20D1DB6813F43C
S31508005930005F1CD1436D23F480734365436D13F4F4
S31508005940805F14D1436D43F0010343650FE0DB68C4
S3150800595013F0020F0BD1436D23F480734365436D37
S3150800596013F4805F03D1436D43F001034365FEF7EB
S3150800597091FB08BD426D12F0100F04D1C26C526B38
S3150800598018469047F5E7FEF799FBF2E708B5806AEF
S31508005990436D43F040034365836D43F00403836519
S315080059A0FEF78CFB08BD0000F0B583B00023019319
S315080059B090F85030012B00F00A8204460D46012368
S315080059C080F8503003689B6813F0040F09D0436DC4
S315080059D043F0200343650120002384F8503003B0C8
S315080059E0F0BD4B68052B08D8023B032B56D8DFE8D9
S315080059F003F0024B4E510C234B602A6869682068F5
S31508005A00FFF744FD2068836813F0040300D00123E0
S31508005A10826812F0080200D001220BB9002A40D091
S31508005A202268936813F0010F17D12B68E868D2F83B
S31508005A30B010C3F3120621EA060100F0180CAA48B2
S31508005A4020FA0CF00340C3F312030B43C2F8B0303C
S31508005A50EA68A64B9A4200F0A9802B68A44A13422A
S31508005A6000F0B181A34A926802F0E070A2498B4225
S31508005A7000F05B81A1498B4200F07E81A0498B42F0
S31508005A8000F08E810020A7E712234B60B5E71823A4
S31508005A904B60B2E74FF480734B60AEE706234B606A
S31508005AA0ABE7AA682968FFF709FD69692268D36820
S31508005AB0C3F3C1035B009940286904280ED02E68F9
S31508005AC0603252F820708F4B3B4006F0F84631435F
S31508005AD00B4343F0004342F82030A1E7136E116EE2
S31508005AE0C1F384612B68C3F3120080BBC3F38463DC
S31508005AF0994234D021684B6E4A6EC2F384622B6891
S31508005B00C3F3120080BBC3F384639A4234D021687E
S31508005B108B6E8A6EC2F384622B68C3F3120080BB55
S31508005B20C3F384639A4234D02168CB6ECA6EC2F33B
S31508005B3084622B68C3F3120080BBC3F384639A4262
S31508005B407FF46EAFCB6E23F00043CB6668E793FA1B
S31508005B50A3F313B1B3FA83F3CAE72023C8E7136E96
S31508005B6023F000431366C5E793FAA3F313B1B3FA18
S31508005B7083F3CAE72023C8E74B6E23F000434B663E
S31508005B80C5E793FAA3F313B1B3FA83F3CAE720235D
S31508005B90C8E78B6E23F000438B66C5E793FAA3F339
S31508005BA013B1B3FA83F3CAE72023C8E720682B6842
S31508005BB0C3F312063EBB9A0E013202F01F02092AEF
S31508005BC08CBF00220122002A55D05EBB990E0131F6
S31508005BD0890601F0F8418EBB4FEA936C0CF1010C73
S31508005BE00CF01F0C012202FA0CF21143AEBB9B0EFD
S31508005BF0013303F01F0303EB43031B051943AA688C
S31508005C00FFF75CFC29E793FAA3F24AB1B2FA82F2EB
S31508005C10013202F01F02092A8CBF00220122D2E7B4
S31508005C202022F5E793FAA3F131B1B1FA81F10131F6
S31508005C30890601F0F841CEE72021F8E793FAA3F2A6
S31508005C404AB1B2FA82F2013202F01F024FF0010C99
S31508005C500CFA02F2C9E72022F5E793FAA3F343B157
S31508005C60B3FA83F3013303F01F0303EB43031B0566
S31508005C70C4E72023F6E7E6B9990E0131890601F053
S31508005C80F84116BB4FEA936C0CF1010C0CF01F0C93
S31508005C90012202FA0CF21143B6BB9B0E013303F044
S31508005CA01F0303EB43031E3B1B0543F00073194315
S31508005CB0A5E793FAA3F131B1B1FA81F10131890669
S31508005CC001F0F841DDE72021F8E793FAA3F24AB19B
S31508005CD0B2FA82F2013202F01F024FF0010C0CFAFE
S31508005CE002F2D8E72022F5E7FFFF070000007F4011
S31508005CF00000088000030450000052C7000084CB4F
S31508005D000100008000F0FF0393FAA3F35BB1B3FA36
S31508005D1083F3013303F01F0303EB43031E3B1B0509
S31508005D2043F00073C3E72023F3E712F4000F7FF470
S31508005D30A1AE2268274B9A4201D000204CE640F4D7
S31508005D40000325498A6822F0E07213438B60234BCF
S31508005D501B689B09224AA2FB03239B09013303EB19
S31508005D6043039B00019302E0019B013B0193019BC6
S31508005D70002BF9D100202FE612F0807F7FF47EAE4B
S31508005D802268144B9A4201D0002025E640F0807321
S31508005D9011498A6822F0E07213438B6000201BE6E3
S31508005DA012F4800F11D122680A4B9A4201D00020C2
S31508005DB012E640F4800308498A6822F0E072134329
S31508005DC08B60002008E6002006E6002004E6022094
S31508005DD005E600BF000004500003045094000020AC
S31508005DE0632D3E0530B583B00023019303689A6896
S31508005DF012F0010F58D1044699682D4A114219D15B
S31508005E009A6822F0004222F03F0242F001029A60AC
S31508005E10284B9B6813F4000F1CD0274B1B689B0963
S31508005E20264AA2FB03239B09013303EB43039B008A
S31508005E3001930CE0436D43F010034365836D43F013
S31508005E4001038365012030E0019B013B0193019B1F
S31508005E50002BF9D1FFF700FB054623681A6812F0F4
S31508005E60010F1FD19A6812F0010F07D19A6822F024
S31508005E70004222F03F0242F001029A60FFF7ECFA74
S31508005E80431B022BE9D923681B6813F0010FE4D1E1
S31508005E90636D43F010036365A36D43F00103A365C7
S31508005EA0012002E0002000E0002003B030BD00BF62
S31508005EB03F0000800003045094000020632D3E0537
S31508005EC070B504460068806810F0040F4ED10E467F
S31508005ED0154694F85030012B4AD0012384F85030E7
S31508005EE02046FFF77FFF00283CD1636D23F47063DB
S31508005EF023F0010343F480736365636D13F4805FD5
S31508005F002DD0A36D23F00603A365E36C194ADA6264
S31508005F10E36C194A1A63E36C184A5A6323681C220D
S31508005F201A60002384F850302268536843F010033F
S31508005F3053602268D36843F00103D36021682B4677
S31508005F4032464031E06C00F091FF2268936823F0F6
S31508005F50004323F03F0343F00403936007E0002364
S31508005F60A365D2E7002384F8503000E0022070BD14
S31508005F700220FCE705590008C55600088D59000897
S31508005F8038B504460268936813F0020300D001236B
S31508005F90916811F0010F39D0002B39D1936803F0BD
S31508005FA00D03012B09D0636D43F010036365A36DE0
S31508005FB043F00103A365012029E0936823F0004319
S31508005FC023F03F0343F002039360236803221A6019
S31508005FD0FFF742FA054623689B6813F0010F13D0B2
S31508005FE0FFF73AFA401B0228F5D923689B6813F095
S31508005FF0010FF0D0636D43F010036365A36D43F0A2
S315080060000103A365012002E0002000E0002038BD5E
S315080060100020FCE730B583B00023019390F8503098
S31508006020012B41D004460D46012380F85030FFF776
S31508006030A7FF80BB636D23F4885323F0020343F064
S31508006040020363652268936823F0404323F03F0305
S3150800605005F080452B4343F00043936023689B6813
S31508006060002B06DB636D23F0030343F0010363652E
S3150800607015E0019B01330193019BB3F5912FEDD3F5
S31508006080636D23F0120343F010036365002384F85D
S315080060905030012006E0636D43F01003636500236A
S315080060A084F8503003B030BD0220FBE770477047D4
S315080060B0704770477047002800F0A18038B504463D
S315080060C090F82030D3B12268136843F001031360B7
S315080060D0FFF7C2F9054623685A6812F0010F10D176
S315080060E0FFF7BAF9401B0A28F5D9636A43F4003367
S315080060F06362052384F82030012038BDFEF776FF59
S31508006100E1E71A6822F002021A60FFF7A5F90546C8
S3150800611023685A6812F0020F0DD0FFF79DF9401B4D
S315080061200A28F5D9636A43F400336362052384F8C1
S3150800613020300120E1E7227E012A3DD01A6822F0AC
S3150800614080021A60637E012B3BD02268136823F015
S3150800615040031360A37E012B39D02268136823F00D
S3150800616020031360E37E012B37D02268136843F0BF
S3150800617010031360237F012B35D02268136823F0A0
S3150800618008031360637F012B33D02268136823F05A
S3150800619004031360A368E268134322691343626920
S315080061A013436268013A21681343CB610020606299
S315080061B0012384F82030A0E71A6842F080021A60AA
S315080061C0C0E72268136843F040031360C2E72268F9
S315080061D0136843F020031360C4E72268136823F0AA
S315080061E010031360C6E72268136843F008031360B8
S315080061F0C8E72268136843F004031360CAE701205E
S315080062007047026890F82030013BDBB2012B05D9B4
S31508006210436A43F4802343620120704730B4D2F8BE
S31508006220003243F00103C2F800324B6903F01F0342
S31508006230012000FA03F3D2F81C026FEA030C20EAE5
S315080062400300C2F81C02C869B0B9D2F80C020CEAFD
S315080062500000C2F80C028C884869CD6844EA0544F7
S31508006260483042F830400C8848698D6844EA05444D
S31508006270483002EBC0004460C86901281BD0886911
S3150800628080BBD2F804020CEA0000C2F804020869CE
S3150800629070BBD2F814020CEA0000C2F81402096AAC
S315080062A001292BD0D2F8003223F00103C2F80032BC
S315080062B0002030BC7047D2F80C021843C2F80C0212
S315080062C08C8848690D6844EA0544483042F83040ED
S315080062D08C8948698D6844EA0544483002EBC00059
S315080062E04460CCE7D2F804021843C2F80402CEE7A9
S315080062F0D2F814021843C2F81402D0E7D2F81C12D6
S315080063000B43C2F81C32CDE770B5044690F820500E
S31508006310EDB2012D06D0436A43F4002343620125FA
S31508006320284670BD022380F820300268136823F0DF
S3150800633001031360FFF790F8064623685B6813F0BD
S31508006340010F0CD0FFF788F8831B0A2BF5D9636A6F
S3150800635043F400336362052384F82030E0E7002520
S315080063606562DDE730B590F820C00468A4680CF1D2
S31508006370FF3C5FFA8CFCBCF1010F62D814F0E05FB9
S3150800638059D0C4F3016C012404FA0CF41C608B6820
S31508006390002B3DD10D68CB68046843EA45550CF1DE
S315080063A018031B01E55003680C690CF1180E03EB82
S315080063B00E135C600B7D012B35D0D17993791B04C4
S315080063C043EA0163517943EA0123147901682343B7
S315080063D001EB0C11C1F88C31D17893781B0443EA90
S315080063E00163517843EA0123117802680B4302EBF3
S315080063F00C12C2F8883102680CF1180C4FEA0C1C12
S3150800640052F80C3043F0010342F80C3000201DE02E
S315080064104C6843EAC403CC6823430CF118042401EE
S3150800642005682B51BFE7036803EB0E13596841F45F
S3150800643080715960C1E7436A43F40013436201203F
S3150800644004E0436A43F480234362012030BD90F898
S3150800645020C00CF1FF3C5FFA8CFCBCF1010F00F286
S31508006460958030B451B90468E46814F0030F10D16C
S31508006470436A43F400134362012077E00468246901
S3150800648014F0030F05D1436A43F400134362012055
S315080064906CE001F11B04240105682C5904F004047E
S315080064A09460002C64D101F11B04240105682C5961
S315080064B0640D1460046801F11B0C4FEA0C1C54F8B7
S315080064C00C4004F00204D46004686444646804F070
S315080064D00F041461046864446468C4F3072494616F
S315080064E0046864446468240C5461026802EB01126F
S315080064F0D2F8B8211A70026802EB0112D2F8B82154
S31508006500C2F307225A70026802EB0112D2F8B821C8
S31508006510C2F307429A70026802EB0112D2F8B82158
S31508006520120EDA70026802EB0112D2F8BC211A7157
S31508006530026802EB0112D2F8BC21C2F307225A7193
S31508006540026802EB0112D2F8BC21C2F307429A7123
S31508006550026802EB0112D2F8BC21120EDA7179B97F
S315080065600268D36843F02003D360002030BC70472C
S3150800657001F11B04240105682C59E408546099E7C5
S315080065800268136943F020031361EEE7436A43F494
S31508006590802343620120704790F82030013BDBB22C
S315080065A0012B05D9436A43F48023436201207047CF
S315080065B0026853690B435361002070477047704760
S315080065C07047704770477047704770477047704705
S315080065D070472DE9F84F054603685C69D3F80480CF
S315080065E09F68D3F80CB0D3F810A0D3F8189014F01D
S315080065F001063BD017F0010616D001229A6017F063
S31508006600020F08D117F0040F0CD117F0080606D0B0
S315080066104FF4805608E0FFF7D1FF002604E0FFF7A5
S31508006620D0FF01E04FF4006617F4807F0DD02B6889
S315080066304FF480729A6017F4007F40F0868017F452
S31508006640806F00F0868046F4005617F4803F0DD020
S315080066502B684FF480329A6017F4003F40F083802D
S3150800666017F4802F00F0838046F4004614F0080FD4
S3150800667007D01BF0100F04D046F400762B681022C2
S31508006680DA6014F0040F02D01BF0080F79D114F069
S31508006690020F04D02B68DB6813F0030F78D114F0CF
S315080066A0400F07D01AF0100F04D046F480662B6806
S315080066B010221A6114F0200F02D01AF0080F6BD1BD
S315080066C014F0100F04D02B681B6913F0030F6AD15E
S315080066D014F4003F02D018F0100F68D114F4803F6C
S315080066E002D018F0080F69D114F4004F7AD018F0C8
S315080066F0040F74D014F4807F04D019F0010F01D070
S3150800670046F0010614F4007F04D019F0020F01D0F8
S3150800671046F0020614F4806F04D019F0040F01D075
S3150800672046F0040614F4006F59D019F0700956D0D3
S31508006730B9F1400F65D058D8B9F1200F5ED0B9F13C
S31508006740300F42D146F0200644E02846FFF737FFCF
S315080067507BE717F4006F02D046F4804675E72846B3
S31508006760FFF730FF71E72846FFF72AFF7EE717F4A1
S31508006770002F02D046F4803678E72846FFF723FF35
S3150800678074E72B680822DA602846FFF71DFF7EE7C4
S315080067902846FDF72BFE82E72B6808221A61284651
S315080067A0FFF714FF8CE72846FFF70FFF90E72B68E3
S315080067B010225A602846FFF70AFF8FE72B6808223F
S315080067C05A602846FFF704FF8EE7B9F1100F01D18A
S315080067D046F008062A68936923F0700393612B68CC
S315080067E004225A609EB9BDE8F88FB9F1500F0BD054
S315080067F0B9F1600FEED146F48076EBE746F0100665
S31508006800E8E746F04006E5E746F08006E2E76B6A09
S3150800681033436B622846FDF70BFEE4E7002807DBE7
S3150800682000F01F02400901239340024A42F8203033
S31508006830704700BF00E100E0002808DB0901C9B283
S3150800684000F1604000F5614080F80013704700F0E1
S315080068500F000901C9B2014B1954704714ED00E045
S3150800686000B500F00700C0F1070CBCF1040F28BF03
S315080068704FF0040C031D062B0FD9C31E4FF0FF3E25
S315080068800EFA0CF021EA000199400EFA03FE22EAFC
S315080068900E0241EA02005DF804FB0023EEE7000061
S315080068A0BFF34F8F0549CA6802F4E062044B1343ED
S315080068B0CB60BFF34F8F00BFFDE700BF00ED00E0E0
S315080068C00400FA05074AD36823F4E0631B041B0C8B
S315080068D0000200F4E060034343F0BF6343F400336F
S315080068E0D360704700ED00E010B50446054BD86844
S315080068F0C0F30220FFF7B4FF01462046FFF79CFFCE
S3150800690010BD00BF00ED00E008B5FFF787FF08BD22
S3150800691008B5FFF7C5FF00000138B0F1807F0BD23C
S315080069204FF0E0235861054AF02182F82310002031
S31508006930986107221A6170470120704700ED00E050
S31508006940002838D010B50446437F1BB3022363776B
S3150800695023791BBB2368194A5A612268936823F076
S3150800696018039360637913BB23684FF0FF321A61EB
S315080069702268936823F0600361690B439360226879
S31508006980936823F08003A1690B439360012363771F
S31508006990002010BD0377FEF77DFBD7E7E268A16804
S315080069A0204600F00DF80028DCD00120F1E7236826
S315080069B022691A61DCE70120704700BFB71DC104D0
S315080069C010B41F231C46013B34B103F01F0C21FAF7
S315080069D00CFC1CF0010FF5D0182A22D8DFE802F0CB
S315080069E00F212121212121211D212121212121219F
S315080069F019212121212121210D00062B15D80368F3
S31508006A00596101688B6823F0180313438B600020D3
S31508006A1008E0072BF3D9012004E00F2BEFD901205A
S31508006A2000E001205DF8044B70470120FAE770B1D9
S31508006A3010B50446037933B102232371002020617F
S31508006A400123237110BD4371FEF73AFBF4E70120D9
S31508006A5070474279012A2CD010B4034601224271AC
S31508006A60022018711C68206801F0100C02FA0CF25A
S31508006A700243226089B919680A6802F03C02042AAE
S31508006A8006D001221A71002058715DF8044B704730
S31508006A904A6842F001024A60F3E719680A6802F494
S31508006AA07012B2F5802FECD14A6842F002024A60B1
S31508006AB0E7E70220704710B483B000240194006809
S31508006AC0019051B901990A4408320192019A13605A
S31508006AD0002003B05DF8044B704701990A4414324C
S31508006AE00192F3E7F8B54379012B00F09480044648
S31508006AF00D46164601234371022303710B68042BC6
S31508006B0032D02B69012B79D02068C16B06F01002B0
S31508006B100723934021EA03012B68AE683343EE68E6
S31508006B20334393400B43C363206803684FF48041A3
S31508006B30914023EA010303602068016840F6FC736C
S31508006B40934021EA03016B6893400B430360206876
S31508006B500368C02101FA02F223EA02030360012353
S31508006B60237100206071F8BDFEF776FC07467EB1FA
S31508006B7023685B6B002B3ADAFEF76EFCC01B012814
S31508006B80F6D9236943F00803236103202071EAE755
S31508006B9023685B6B13F4004F0BD0FEF75DFCC01B3C
S31508006BA00128F5D9236943F00803236103202071DE
S31508006BB0D9E70120FEF756FC2368AA691A642068FB
S31508006BC0836C06F0100240F2FF31914023EA01037C
S31508006BD0E96991400B4383642068C36CFF219140A7
S31508006BE023EA0103296A91400B43C36489E701201C
S31508006BF0FEF738FC2368AA695A64E0E721688A6BBD
S31508006C0006F010001F23834022EA03026B698340C3
S31508006C1013438B6378E70220A5E7002800F08380FA
S31508006C202DE9F04F83B0894604460379DBB2022B7F
S31508006C307BD04379012B7AD0012141710068C56B5D
S31508006C4002F010070723BB4005EA030B0568B940A5
S31508006C5025EA010101602068C16B6FEA030A21EA8F
S31508006C600303C3632368019392B9019B0833019315
S31508006C70019B4FF400621A60226813684FF480483B
S31508006C8008FA07F843EA080313600825102605E002
S31508006C90019B14330193EBE72E446D089DB12168DF
S31508006CA08B6B1F22BA4023EA020306FA07F2134344
S31508006CB08B630120FEF7D6FB23685B6B38EA030378
S31508006CC0EAD1761BE9E721688B6B1F22BA40D543C8
S31508006CD023EA020306FA07F213438B630120FEF741
S31508006CE0C1FB23685A6B18EA020F06D101369A6B64
S31508006CF0154006FA07F73D439D632268136823EAA1
S31508006D0008031360C9F814600123C9F81030226813
S31508006D10D36B0AEA030A4AEA0B03D36300206071BD
S31508006D2003B0BDE8F08F012070470120F8E7022084
S31508006D30F6E730B4446C04F01C0C012404FA0CF495
S31508006D40056C6C60046863608368102B05D0036863
S31508006D5099600368DA6030BC704703689A60036814
S31508006D60D960F8E7002873D010B403460068394A9A
S31508006D7090424AD8384A02443849A1FB02121209FD
S31508006D8092005A64364A1A64022283F8252001685A
S31508006D9021F4FF4121F070019A68DC6822431C69DE
S31508006DA022435C6922439C692243DC6922431C6AAC
S31508006DB022430A4302609A68B2F5804F1BD0196CC9
S31508006DC0274A91422CD0264AD2F8A814586C00F0CB
S31508006DD01C0C0F2000FA0CF021EA0001C2F8A814D6
S31508006DE0D2F8A81458685C6C04F01C0C00FA0CF075
S31508006DF00143C2F8A8140020D863012283F825208D
S31508006E0083F824005DF8044B7047164A0244134978
S31508006E10A1FB0212120992005A64134A1A64B3E7D4
S31508006E20D2F8A810586C00F01C0C0F2000FA0CF0D1
S31508006E3021EA0001C2F8A810D2F8A81058685C6CBC
S31508006E4004F01C0C00FA0CF00143C2F8A810D2E7B3
S31508006E500120704707040240F8FFFDBFCDCCCCCC1B
S31508006E6000000240F8FBFDBF0004024038B50446A6
S31508006E7090F82400012832D0012084F8240094F8E0
S31508006E802500C0B2012804D0002384F8243002204B
S31508006E9038BD022084F825000020E06325682868AC
S31508006EA020F0010028602046FFF743FF236B5BB103
S31508006EB02268136843F00E0313602268136843F0D0
S31508006EC0010313600020E3E72268136823F0040334
S31508006ED013602268136843F00A031360EDE7022083
S31508006EE0D6E708B590F82530DBB2022B03D0042389
S31508006EF0C363012008BD0268136823F00E031360FC
S31508006F000268136823F001031360436C03F01C0343
S31508006F10016C012202FA03F34B6080F82520002356
S31508006F2080F82430836B13B198470020E2E70020ED
S31508006F30E0E738B5036C196804682568436C03F004
S31508006F401C0304229A400A4215D015F0040F12D0E9
S31508006F50236813F0200F03D1236823F0040323606A
S31508006F60436C03F01C02016C042393404B60036BD3
S31508006F7003B1984738BD02229A400A421CD015F040
S31508006F80020F19D0236813F0200F06D1236823F0C7
S31508006F900A032360012380F82530436C03F01C02A2
S31508006FA0016C022393404B60002380F82430C36AA7
S31508006FB0002BDFD09847DDE7082202FA03F30B42DD
S31508006FC0D8D015F0080FD5D0236823F00E03236018
S31508006FD0436C03F01C03016C012202FA03F34B60B5
S31508006FE0C26380F82520002380F82430436B002BE9
S31508006FF0C0D09847BEE7000010B4064C616941F05E
S31508007000010161610260BFF36F8F43605DF8044B55
S31508007010704700BF00200240094A536943F48023A1
S315080070205361EFF3108C72B6402351F8042B40F8E5
S31508007030042B013B13F0FF03F7D18CF3108870473C
S3150800704000200240094B5B69002B01DB00207047DA
S31508007050064B074A9A6002F188329A605B69002BF0
S3150800706001DB002070470120704700BF0020024066
S3150800707023016745034A536943F0004353610020DF
S31508007080704700BF0020024038B50446FEF7E4F911
S315080070900546144B1B6913F4803F09D0B4F1FF3F32
S315080070A0F7D0FEF7D9F9401BA042F2D3032015E02A
S315080070B00C4B1B690C4A134009D10A4B1B6913F088
S315080070C0010F0CD0074B01221A61002006E0074980
S315080070D04A681A434A60034A1361012038BD0020F2
S315080070E0FCE700BF00200240FAC30200A00000200F
S315080070F02DE9F0411646284A1278012A49D0044655
S315080071000D469846244B01221A704CF25030FFF770
S31508007110BBFF074608BB204B00225A601F4B1B6863
S3150800712013F4806F1FD01D4A136823F4806313601D
S31508007130194B02221A77D4B1631E012B1ED90024DB
S315080071404CF25030FFF7A0FF074624B1134A5369A3
S3150800715023EA0403536100F047F80F4B00221A7024
S315080071603846BDE8F0810C4B00221A77E3E7324631
S3150800717043462846FFF740FF0124E1E73146284603
S31508007180FFF74AFF022C01D00024D9E74FF48024E8
S31508007190D6E70227E4E700BFA0000020002002404F
S315080071A010F0010F04D0054A536943F004035361F4
S315080071B0024A536943F48033536170470020024002
S315080071C0084B5A6922F47E72C00000F4FF6002433D
S315080071D05A615A6942F002025A615A6942F4803287
S315080071E05A61704700200240164B1B7FDBB2012B09
S315080071F001D0032B10D1144A116821F400711160D3
S31508007200116841F400611160116821F40061116090
S31508007210116841F400711160023BDBB2012B03D9FE
S31508007220084B00221A777047074B1A6842F48052B7
S315080072301A601A6822F480521A601A6842F4806248
S315080072401A60EDE7A000002000200240F8B5394B8F
S315080072501B78012B6BD004460E46364B01221A705A
S315080072604CF25030FFF710FF074600285AD1314B31
S3150800727000225A60304B1B6813F4007F2FD02E4B28
S315080072801B6813F4806F26D02B4A136823F4806397
S315080072901360284B03221A772368012B31D04FF04D
S315080072A0FF333360A568A368E2681344AB4237D955
S315080072B061682846FFF784FF4CF25030FFF7E4FE7A
S315080072C01D4A536923F47E7323F00203536107466C
S315080072D028BB0135E7E7174B01221A77DCE7164B7F
S315080072E01B6813F4806F08D0134A136823F480636D
S315080072F01360104B02221A77CEE70E4B00221A773C
S31508007300CAE76068FFF74CFF4CF25030FFF7BCFE47
S315080073100746094A536923F00403536100E03560C0
S31508007320FFF762FF034B00221A703846F8BD0227A2
S31508007330FBE700BFA000002000200240F0B583B0A4
S31508007340002362E085685E000324B44025EA04054C
S31508007350CC68B4402C438460456825EA0C054C6823
S31508007360C4F300149C402C4344605FE0DD080835F4
S3150800737050F8254003F0070C4FEA8C0C4FF00F0E1F
S315080073800EFA0CFE24EA0E0E0C6904FA0CF444EA12
S315080073900E0440F8254060E0022400E0002404FAC8
S315080073A00EF42C430CF1020C4C4D45F82C404C4C79
S315080073B0A568D44325EA02064F6817F4801F01D052
S315080073C042EA0506464DAE60ED6804EA05064F68D2
S315080073D017F4001F01D042EA0506414DEE606D68BC
S315080073E004EA05064F6817F4003F01D042EA05068D
S315080073F03B4D6E602D682C404E6816F4803F01D0D8
S3150800740042EA0504364A146001330A6832FA03F47C
S3150800741062D04FF0010C0CFA03FC1CEA0202F3D00E
S315080074204C6804F00304013C012C8BD94C6804F029
S315080074300304032C0CD0C4685D004FF0030C0CFA4F
S3150800744005FC24EA0C0C8C68AC4044EA0C04C460C5
S315080074504C6804F00304022C88D004684FEA430EF3
S315080074604FF0030C0CFA0EFC24EA0C0C4C6804F0E2
S31508007470030404FA0EF444EA0C0404604C6814F499
S31508007480403FC1D0174C256E45F001052566246E90
S3150800749004F001040194019C4FEA930C0CF10205D7
S315080074A00E4C54F8255003F0030E4FEA8E0E0F24A7
S315080074B004FA0EF425EA0405B0F1904F3FF46EAFD6
S315080074C0094CA04206D004F58064A0423FF464AF9C
S315080074D0072464E7012462E703B0F0BD0000014019
S315080074E000040140001002400004004803691942E4
S315080074F001D001207047002070470AB181617047AA
S3150800750081627047436901EA030221EA030141EAFD
S31508007510024181617047002859D010B5044690F899
S315080075204130002B43D0242384F841302268136865
S3150800753023F0010313606368226823F07063136104
S315080075402268936823F400439360E368012B33D0E1
S31508007550A368226843F404439360E368022B31D09E
S315080075602268536843F0007343F40043536022686B
S31508007570D36823F40043D360236962691343A1697E
S31508007580226843EA0123D360E369216A22680B4330
S3150800759013602268136843F00103136000206064D7
S315080075A0202384F84130206384F8420010BD80F817
S315080075B04030FDF7B5FDB6E7A368226843F40043FB
S315080075C09360CAE723684FF400625A60C8E701204F
S315080075D07047034690F84120D2B2202A23D190F86A
S315080075E04020012A21D0012280F84020242280F858
S315080075F041200068026822F00102026018680268E9
S3150800760022F4805202601868026811430160196802
S315080076100A6842F001020A60202283F8412000200D
S3150800762083F84000704702207047022070470346DF
S3150800763090F84120D2B2202A21D190F84020012A80
S315080076401FD0012280F84020242280F841200068BB
S31508007650026822F0010202601868026822F4706269
S3150800766042EA0122026019680A6842F001020A60C9
S31508007670202283F84120002083F84000704702202A
S3150800768070470220704700282FD038B50446036893
S315080076904CF6CC421A60036845F255521A600368E4
S315080076A042685A60036882689A60FDF7D5FE054607
S315080076B02368DA6812F0070F0BD0FDF7CDFE401BE2
S315080076C03128F5D92368DB6813F0070FF0D00320BB
S315080076D005E01969E268914202D01A61002038BDB6
S315080076E04AF6AA221A600020F9E7012070470368C3
S315080076F04AF6AA221A60002070470000024B186852
S3150800770000F4C060704700BF00700040B0F5007F0D
S315080077100FD01F4B1B6803F4C063B3F5806F34D0DA
S315080077201B4A136823F4C06343F480631360002084
S315080077307047174B1B6803F4C063B3F5007F20D06E
S31508007740134A136823F4C06343F400731360114BA0
S315080077501B68322202FB03F30F4AA2FB03239B0C8E
S31508007760013300E0013B0A4A526912F4806F01D0E6
S31508007770002BF7D1064B5B6913F4806F03D1002009
S31508007780704700207047032070470020704700BFED
S31508007790007000409400002083DE1B4330B583B0A0
S315080077A00446204B9B6D13F0805F0BD0FFF7A6FFB6
S315080077B0B0F5007F17D0802C1FD82DD0702C2DD077
S315080077C000211BE0174DAB6D43F08053AB65AB6DE5
S315080077D003F080530193019BFFF790FFAB6D23F0F5
S315080077E08053AB65E4E7802C03D9A02C03D902218A
S315080077F004E0002102E0012100E003210A4A13689F
S3150800780023F007030B431360136803F007038B4247
S3150800781006D1002003B030BD0221EFE70121EDE7D4
S315080078200120F7E70010024000200240284A93682A
S31508007830D26802F0030213F00C030AD00C2B06D010
S31508007840042B1FD0082B20D00020024610E0012A66
S31508007850F6D11F4A126812F0080F0CD11C4AD2F84A
S315080078609420C2F303221B4951F8222043B1002079
S315080078700C2B0DD07047164A1268C2F30312F2E7B2
S315080078801046F5E714480022F2E714480022EFE70D
S315080078900F4BDB6803F00303022B16D0032B00D132
S315080078A00E4A0B49CB68C3F302130133C868C0F309
S315080078B0062002FB00F0B0FBF3F0CB68C3F341638C
S315080078C001335B00B0FBF3F0D4E7034AE9E700BFF6
S315080078D0001002401CD200080024F400005A62027C
S315080078E0002800F01C83F0B583B00446964B9D68CB
S315080078F005F00C05DE6806F00306036813F0100FA2
S315080079005AD0E5B10C2D18D0A369002B00F0BB8026
S315080079108D4A136843F001031360FDF79DFD074682
S31508007920894B1B6813F0020F40F09A80FDF794FD0F
S31508007930C01B0228F4D90320FCE2012EE4D1824BB5
S315080079401B6813F0020F03D0A369002B00F0E9822D
S31508007950206A7D4B1B6813F0080F5BD07A4B1B68B7
S3150800796003F0F00398425CD8774B1A6842F0080295
S315080079701A601A6822F0F002216A0A431A605A68E5
S3150800798022F47F42E16942EA01225A60002D60D062
S31508007990FFF74CFF6C4B9B68C3F303136B4AD35C2E
S315080079A003F01F03D8406A4B18606A4B1868FDF746
S315080079B00FFD002840F0BE82236813F0010F00F087
S315080079C08180082D75D00C2D71D06368B3F5803F82
S315080079D000F09780B3F5A02F00F099805A4B1A68EB
S315080079E022F480321A601A6822F480221A606368C8
S315080079F0002B00F09980FDF72FFD0746524B1B68B8
S31508007A0013F4003F5ED1FDF727FDC01B6428F5D9A6
S31508007A1003208FE24C4BD3F894301B0903F0F00394
S31508007A20A0E7FFF7BBFE002840F07D82464B1A68A8
S31508007A3042F008021A601A6822F0F002216A0A4324
S31508007A401A605A6822F47F42E16942EA01225A60C2
S31508007A509EE7206AFFF7A2FE002899D0012069E276
S31508007A60394B1A6842F008021A601A6822F0F002C6
S31508007A70216A0A431A605A6822F47F42E16942EA97
S31508007A8001225A6098E7304A136823F0010313600D
S31508007A90FDF7E2FC07462C4B1B6813F0020F8BD050
S31508007AA0FDF7DAFCC01B0228F5D9032042E2032EB3
S31508007AB08BD1254B1B6813F4003F03D06368002B5A
S31508007AC000F03382236813F0020F58D0042D45D0F6
S31508007AD00C2D41D0E368002B77D01B4A136843F47A
S31508007AE080731360FDF7B8FC0646174B1B6813F442
S31508007AF0806F61D1FDF7B0FC801B0228F5D9032001
S31508007B0018E2114A136843F4803313606FE703F1F0
S31508007B108043A3F53C331A6842F480221A601A6837
S31508007B2042F480321A6062E7FDF796FC0746064B78
S31508007B301B6813F4003FC5D0FDF78EFCC01B6428F4
S31508007B40F5D90320F6E100BF001002404CD2000828
S31508007B50940000209C000020022EBBD1A44B1B6879
S31508007B6013F4806F03D0E368002B00F0E081A04A8D
S31508007B70536823F0F853216943EA01635360236885
S31508007B8013F0080F4CD063699BB3994AD2F8943026
S31508007B9043F00103C2F89430FDF75EFC0646944BA9
S31508007BA0D3F8943013F0020F3AD1FDF755FC801B39
S31508007BB00228F4D90320BDE18D4A536823F0F8530F
S31508007BC0216943EA01635360D9E7894A136823F4B4
S31508007BD080731360FDF740FC0646854B1B6813F45B
S31508007BE0806FCCD0FDF738FC801B0228F5D903201E
S31508007BF0A0E17F4AD2F8943023F00103C2F894300A
S31508007C00FDF72AFC06467A4BD3F8943013F0020F98
S31508007C1006D0FDF721FC801B0228F4D9032089E150
S31508007C20236813F0040F7AD0714B9B6D13F0805FB5
S31508007C3036D16F4B9A6D42F080529A659B6D03F070
S31508007C4080530193019B01266A4B1B6813F4807FBE
S31508007C5028D0A368012B39D0052B3FD0644BD3F825
S31508007C60902022F00102C3F89020D3F8902022F049
S31508007C700402C3F89020A368002B3DD0FDF7ECFB67
S31508007C8007465B4BD3F8903013F0020F46D1FDF749
S31508007C90E3FBC01B41F288339842F2D9032049E13D
S31508007CA00026D1E7534A136843F480731360FDF73F
S31508007CB0D3FB07464F4B1B6813F4807FC9D1FDF7EA
S31508007CC0CBFBC01B0228F5D9032033E1484AD2F87A
S31508007CD0903043F00103C2F89030CCE7444BD3F818
S31508007CE0902042F00402C3F89020D3F8902042F086
S31508007CF00102C3F89020BEE7FDF7AEFB07463C4BF2
S31508007D00D3F8903013F0020F08D0FDF7A5FBC01B7F
S31508007D1041F288339842F2D903200BE1E6B9236889
S31508007D2013F0200F35D0636AE3B1314AD2F89830A0
S31508007D3043F00103C2F89830FDF78EFB06462C4B3C
S31508007D40D3F8983013F0020F23D1FDF785FB801B7B
S31508007D500228F4D90320EDE0254A936D23F08053D9
S31508007D609365DCE7224AD2F8983023F00103C2F87B
S31508007D709830FDF771FB06461D4BD3F8983013F083
S31508007D80020F06D0FDF768FB801B0228F4D90320F2
S31508007D90D0E0A36A002B00F0CC80022B17D00C2D64
S31508007DA000F0CC80124A136823F080731360FDF745
S31508007DB053FB04460E4B1B6813F0007F00F0A880A7
S31508007DC0FDF74AFB001B0228F4D90320B2E0084B52
S31508007DD0DB6803F00301E26A91420DD00C2D00F036
S31508007DE0AB80034B1B6813F0806F2FD00120A1E0F6
S31508007DF0001002400070004003F07002216B013948
S31508007E00B2EB011FEAD103F4FE42616BB2EB012F1C
S31508007E10E4D103F07842A16BB2EBC16FDED103F473
S31508007E20C001E26B5208013AB1EB425FD6D103F0CA
S31508007E30C063226C5208013AB3EB426FCED1404B75
S31508007E401B6813F0007F49D0002073E03C4A136892
S31508007E5023F080731360FDF7FFFA0546384B1B685D
S31508007E6013F0007F06D0FDF7F7FA401B0228F5D974
S31508007E7003205FE0324AD36832491940E36A206B2F
S31508007E80013843EA0013606B43EA0023E06B4008BD
S31508007E90013843EA4053206C4008013843EA4063FE
S31508007EA0A06B43EAC0631943D160136843F080733B
S31508007EB01360D36843F08073D360FDF7CDFA0446A8
S31508007EC01F4B1B6813F0007F06D1FDF7C5FA001B90
S31508007ED00228F5D903202DE000202BE0184B1A685C
S31508007EE042F080721A60DA6842F08072DA60FDF752
S31508007EF0B3FA0446124B1B6813F0007F06D1FDF750
S31508007F00ABFA031B022BF5D9032013E0002011E07E
S31508007F100B4AD1680C4B0B40D36000200AE00120C5
S31508007F207047012006E0012004E0012002E001205C
S31508007F3000E0002003B0F0BD0120FBE70120F9E7CF
S31508007F40001002408C809D01FCFFEEFE002800F028
S31508007F50AF8070B50D460446594B1B6803F00703FE
S31508007F608B420BD2564A136823F007030B43136060
S31508007F70136803F007038B4240F09C80236813F0D4
S31508007F80020F0CD0A2684F4B9B6803F0F0039A428D
S31508007F9005D94C498B6823F0F0031A438A60236895
S31508007FA013F0010F39D06368032B09D0022B26D0B2
S31508007FB063BB444A126812F0020F06D1012076E02C
S31508007FC0404A126812F0007F76D03E498A6822F04D
S31508007FD0030213438B60FDF73FFA0646394B9B684D
S31508007FE003F00C036268B3EB820F16D0FDF734FA80
S31508007FF0801B41F288339842F0D9032057E0314A72
S31508008000126812F4003FE0D1012050E02D4A1268B0
S3150800801012F4806FD9D1012049E0236813F0020FCA
S315080080200CD0A268274B9B6803F0F0039A4205D24E
S3150800803024498B6823F0F0031A438A60204B1B6897
S3150800804003F00703AB420AD91D4A136823F0070356
S315080080502B431360136803F00703AB422ED1236842
S3150800806013F0040F06D0174A936823F4E063E16817
S315080080700B439360236813F0080F07D0114A9368DF
S3150800808023F46053216943EAC1039360FFF7CEFBEB
S315080080900C4B9B68C3F303130B4AD35C03F01F0313
S315080080A0D8400A4B18600A4B1868FDF791F970BD5D
S315080080B0012070470120FAE70120F8E70120F6E7DA
S315080080C000200240001002404CD200089400002014
S315080080D09C000020F8B504460D46584BDB6813F0A3
S315080080E0030F17D0554BDB6803F00303026893426E
S315080080F001D0012616E0002A00F09E804F4BDB686F
S31508008100C3F3021301334268934201D0012609E002
S3150800811000261BE00368022B57D0032B5CD0012BEB
S3150800812002D001263046F8BD444A126812F0020F02
S315080081305ED04248C26822F073026168013943EA98
S3150800814001131343C3600026002EEBD13B4A136884
S3150800815023F080631360FDF77FF90746374B1B68EA
S3150800816013F0006F05D0FDF777F9C31B022BF5D97D
S315080081700326002ED6D1002D3CD130490B6923F0B9
S31508008180784323F4FE43A068E268D20642EA002256
S3150800819013430B61294A136843F080631360FDF7A4
S315080081A05BF90546254B1B6813F0006F05D1FDF7F3
S315080081B053F9401B0228F5D90326002EB2D11F4ACF
S315080081C01369A1690B431361ACE71C4A126812F4E0
S315080081D0806FAED10126A5E7184A126812F4003F4F
S315080081E0A7D1164A126812F4802FA2D1012699E760
S315080081F00126A9E7012D0FD01048026922F0C062B6
S3150800820022F4FE42A16863695B08013B5B0643EA08
S3150800821001231A430261BDE70848026922F4C00235
S3150800822022F4FE42A16823695B08013B5B0543EA29
S3150800823001231A430261ADE7012673E700100240E5
S315080082402DE9F04182B00446036813F4006F25D087
S31508008250C36BB3F5000F06D0B3F5400F12D04BB180
S31508008260012637461CE0AE4AD36843F48033D36010
S31508008270002708E000210430FFF72CFF074610B15D
S3150800828006460DE00027A64AD2F8883023F44003B4
S31508008290E16B0B43C2F88830002601E0002637461A
S315080082A0236813F4003F6BD09D4B9B6D13F0805FE2
S315080082B04CD19B4B9A6D42F080529A659B6D03F0A8
S315080082C080530193019B4FF00108964A136843F4C3
S315080082D080731360FDF7C0F80546924B1B6813F4CC
S315080082E0807F05D1FDF7B8F8401B0228F5D903278A
S315080082F0002F40D18A4BD3F8903013F4407315D031
S31508008300226D9A4212D0864AD2F8903023F44073EE
S31508008310D2F8901041F48031C2F89010D2F890103B
S3150800832021F48031C2F89010C2F8903013F0010F92
S315080083300FD1002F40F0C980794AD2F8903023F443
S315080083404073216D0B43C2F8903015E04FF00008DA
S31508008350BBE7FDF781F80546714BD3F8903013F06B
S31508008360020FE6D1FDF778F8401B41F288339842B0
S31508008370F2D90327DDE73E46B8F1000F40F0A780A3
S31508008380236813F0010F08D0654AD2F8883023F025
S315080083900303216A0B43C2F88830236813F0020FDF
S315080083A008D05F4AD2F8883023F00C03616A0B4381
S315080083B0C2F88830236813F0200F08D0584AD2F83C
S315080083C0883023F44063A16A0B43C2F888302368D7
S315080083D013F4007F08D0524AD2F8883023F4402399
S315080083E0616B0B43C2F88830236813F4806F08D09A
S315080083F04B4AD2F8883023F44013A16B0B43C2F8DA
S315080084008830236813F0400F08D0454AD2F88830E0
S3150800841023F44053E16A0B43C2F88830236813F407
S31508008420807F08D03E4AD2F8883023F44033216B47
S315080084300B43C2F88830236813F4005F0FD0384A1C
S31508008440D2F8883023F04063216C0B43C2F8883099
S31508008450236CB3F1006F40D0B3F1806F42D023682C
S3150800846013F4802F0FD02E4AD2F8883023F04063B9
S31508008470616C0B43C2F88830636CB3F1006F39D076
S31508008480B3F1806F3BD0236813F4804F0CD0244A95
S31508008490D2F8883023F04053A16C0B43C2F88830D9
S315080084A0A36CB3F1805F32D0236813F4004F08D071
S315080084B01B4AD2F8883023F08043E16C0B43C2F89C
S315080084C08830304602B0BDE8F0813E4654E7144A8B
S315080084D0936D23F08053936552E7D36843F4801372
S315080084E0D360BCE70121201DFFF7F4FD0028B6D0B4
S315080084F00646B4E7D36843F48013D360C3E7012183
S31508008500201DFFF7E7FD0028BDD00646BBE7022180
S31508008510201DFFF7DFFD0028C6D00646C4E700BFCA
S3150800852000100240007000402DE9F04782B0054671
S31508008530884617461E46FCF78FFF0A9B1B1A03EB55
S315080085400609FCF789FF8246284B1B68C3F3CB3321
S3150800855009FB03F301932B689C6838EA04040CBFF3
S3150800856001230023BB423DD0B6F1FF3FF3D0FCF711
S3150800857073FFA0EB0A00484507D2019A02B14A46A2
S31508008580019B013B01939146E5E72A68536823F06E
S31508008590E00353606B68B3F5827F0BD0AB6AB3F523
S315080085A0005F14D0012385F85D30002385F85C3020
S315080085B0032018E0AB68B3F5004F02D0B3F5806F1F
S315080085C0ECD12A68136823F040031360E6E72A68AB
S315080085D0136823F4005313602A68136843F400539E
S315080085E01360DFE7002002B0BDE8F08794000020A2
S315080085F02DE9F04782B006460C4615461F4600236D
S315080086008DF80330FCF728FF0A9B1B1A03EB0708B3
S31508008610FCF722FF8146D6F800A0304B1B6803EB17
S315080086208303C3EBC3031B0D08FB03F3019302E0AB
S31508008630B7F1FF3F12D133689B6803EA040CAC45D7
S3150800864047D0B4F5C06FF3D1002DF1D19AF80C30AC
S31508008650DBB28DF803309DF80330E9E7FCF7FCFE42
S31508008660A0EB0900404507D2019A02B14246019B98
S31508008670013B01939046DEE73268536823F0E00336
S3150800868053607368B3F5827F0BD0B36AB3F5005FA6
S3150800869014D0012386F85D30002386F85C30032069
S315080086A018E0B368B3F5004F02D0B3F5806FECD18C
S315080086B03268136823F040031360E6E732681368EC
S315080086C023F4005313603268136843F400531360AD
S315080086D0DFE7002002B0BDE8F08700BF9400002065
S315080086E070B582B004460D46164600920B46002227
S315080086F04FF4C051FFF77CFFB0B900962B46002215
S3150800870080212046FFF710FFA8B900962B460022C5
S315080087104FF4C0612046FFF76BFF50B1236E43F05C
S3150800872020032366032004E0236E43F02003236618
S31508008730032002B070BD236E43F020032366032096
S31508008740F7E770B582B004460D4616464368B3F59A
S31508008750827F0DD000962B46002280212046FFF707
S31508008760E3FE90B96368B3F5827F14D002B070BD9A
S315080087708368B3F5004F02D0B3F5806FEAD122685B
S31508008780136823F040031360E4E7236E43F02003E5
S3150800879023660320EAE7A368B3F5004F02D0B3F5D2
S315080087A0806FE3D100962B4600224FF4C061204625
S315080087B0FFF71EFF0028D9D0236E43F02003236657
S315080087C00320D3E700286AD010B50446436A33B9B4
S315080087D04368B3F5827F05D00023C36102E0002316
S315080087E0036143610023A36294F85D30002B4DD0EA
S315080087F0022384F85D302268136823F0400313606F
S31508008800E368B3F5E06F47D90022B3F5706F04D07B
S31508008810B3F5E06F01D00023A362636803F48273A3
S31508008820A16801F404410B43216901F002010B43DD
S31508008830616901F001010B43A16901F400710B4361
S31508008840E16901F038010B43216A01F080010B430D
S31508008850A16A01F4005120680B430360638B03F09F
S315080088600403616A01F010010B43616B01F0080112
S315080088700B43E16801F470610B4321681A434A60AF
S3150800888000202066012384F85D3010BD84F85C3032
S315080088902046FCF789FCABE74FF48052B5E7012088
S315080088A07047000038B5044690F85C00012800F0CF
S315080088B0F780012084F85C0094F85D00C0B2656812
S315080088C001280AD0B5F5827F40F0DB80A568002D27
S315080088D040F0DC80042840F0DB80002900F0DA80D4
S315080088E0002A00F0D980002B00F0D88094F85D00AB
S315080088F0C0B2042802D0052084F85D000020206656
S31508008900A163A387E3872264A4F84430A4F8463019
S31508008910E06420652268536823F4C0435360E36823
S31508008920B3F5E06F28D92268536823F4805353605F
S3150800893094F85D30DBB2042B69D0A36D594A1A63EB
S31508008940A36D594ADA62A36D584A5A63A36D002289
S315080089509A632168B4F846309BB2226C0C31A06D3C
S31508008960FEF784FA002859D0236E43F010032366D5
S31508008970012084F85D0085E02268536843F480533B
S315080089805360636D9B69B3F5806F1AD0A36D9B69BD
S31508008990B3F5806FCCD12268536823F480535360B3
S315080089A0B4F8463013F0010F24D12268536823F433
S315080089B000535360B4F84630C3F34E03A4F8463068
S315080089C0B6E7A38F13F0010F09D12268536823F481
S315080089D080435360E38FC3F34E03E387D6E72268E9
S315080089E0536843F480435360E38FC3F34E03013364
S315080089F0E387CBE72268536843F400535360B4F81F
S31508008A004630C3F34E030133A4F8463090E7A36D0E
S31508008A10274A1A63A36D274ADA6294E722685368DD
S31508008A2043F001035360626D00231363626DD362E2
S31508008A30626D5363626D93632268E38F9BB20C3257
S31508008A40A16B606DFEF712FA98B923681A6812F0DE
S31508008A50400F03D11A6842F040021A602268536830
S31508008A6043F0200353602268536843F002035360BF
S31508008A7008E0236E43F010032366012084F85D00A6
S31508008A8000E00220002384F85C3038BD0220F9E7B4
S31508008A900220F7E70120F5E70120F3E70120F1E7D7
S31508008AA00220F2E7C78A0008638B0008D18A00080B
S31508008AB0BB8A0008F38A0008704708B5806AFFF782
S31508008AC0FBFF08BD704708B5806AFFF7FBFF08BDC6
S31508008AD008B5806A0268536823F003035360036E7F
S31508008AE043F010030366012380F85D30FBF700FEB0
S31508008AF008BD38B50546846AFCF7AEFC2B681B68CA
S31508008B0013F0200F1FD1024621684B6823F020037B
S31508008B104B60A3681BB96368B3F5827F17D02168D9
S31508008B204B6823F001034B6064212046FFF709FEDA
S31508008B3008B1202323660023A4F84630012384F8CD
S31508008B405D30236E4BB92046FBF7C0FD38BD216862
S31508008B504B6823F003034B60E6E72046FBF7C8FDA6
S31508008B60F4E738B50546846AFCF776FC2B681B687B
S31508008B7013F0200F1CD1024621684B6823F020030E
S31508008B804B6064212046FFF7ABFD18B1236E43F016
S31508008B90200323662268536823F0030353600023E7
S31508008BA0E387A4F84630012384F85D30236E1BB9A9
S31508008BB02046FBF779FD38BD2046FBF799FDFAE715
S31508008BC010B584B0044602685168936803F0410002
S31508008BD0012867D013F0020F02D011F0800F68D178
S31508008BE013F4B07F68D011F0200F65D013F0400F52
S31508008BF00FD094F85D00C0B203285FD0206E40F015
S31508008C000400206600200090D068009090680090CC
S31508008C10009813F0200F0CD0206E40F0010020665B
S31508008C200020029090680290106820F040001060C2
S31508008C30029A13F4807F09D0236E43F00803236653
S31508008C400023039323689B680393039B236E002BDF
S31508008C5032D02268536823F0E0035360012384F876
S31508008C605D3011F0030F31D02268536823F00303F7
S31508008C705360A36D4BB1174A9A63A06DFEF731F99D
S31508008C8018B1236E43F040032366636DA3B1114AFE
S31508008C909A63606DFEF725F970B1236E43F04003C1
S31508008CA0236609E011F0400F94D0E36C20469847FC
S31508008CB002E0236D2046984704B010BD00230193B7
S31508008CC0D368019393680193019BF5E72046FBF768
S31508008CD00FFDF1E7D98C000808B5806A0023A0F8D3
S31508008CE04630C387FBF704FD08BD844600231120E0
S31508008CF08B4212D230B402E008338B420BD203EB1C
S31508008D000C02D2E90045B5F1FF3F08BFB4F1FF3FB9
S31508008D10F2D01020F0E730BC704770472DE9F00319
S31508008D20D0E90089D0E90267D0E90445D0E90623ED
S31508008D30B3F1FF3F08BFB2F1FF3F13D1B5F1FF3FD3
S31508008D4008BFB4F1FF3F11D1B7F1FF3F08BFB6F135
S31508008D50FF3F0DD1B9F1FF3F08BFB8F1FF3F09D179
S31508008D60002000E00420BDE8F00370470320FAE77E
S31508008D700220F8E70120F6E738B5044600F5803CFE
S31508008D804FEACC2C284BD3F8E02590B24FF6FF7368
S31508008D90984215D0254B03EA82234FF4F032B2FBF2
S31508008DA0F3F203FB02CC0CF108050CF110000CF1F0
S31508008DB0180E0139032931D8DFE801F005101B2503
S31508008DC04FF48023E9E74FF0AA324FF0AA33604602
S31508008DD000F08AFF20BB164B1C7038BD4FF0AA3234
S31508008DE04FF0AA33284600F07FFFD8B9104B1C7005
S31508008DF0F3E74FF0AA324FF0AA3300F075FF0028C8
S31508008E00EBD00220E9E74FF0AA324FF0AA337046BA
S31508008E1000F06AFF0028E0D00220DEE70020DCE749
S31508008E200220DAE70220D8E70070FF1F00FCFF03E4
S31508008E30E004002038B5054600F088FF002840F019
S31508008E4092804B4BD3F8E02591B24FF6FF739942C7
S31508008E500CD0484B03EA82234FF4F034B4FBF3F406
S31508008E6003FB04F4C4F5F034E40A13E04FF480235A
S31508008E70F2E704F580304FF4F033B3FBF2F302FB6C
S31508008E8003F34FF4006103EBC020FFF72EFF102811
S31508008E9021D00134364BD3F8E03599B24FF6FF723C
S31508008EA0914220D0334A02EA83224FF4F033B3FBCF
S31508008EB0F2F302FB03F3C3F5F033DB0A0433A342F0
S31508008EC014D9002DD5D10121204600F019FF00281C
S31508008ED0DFD0012040E00121204600F011FF0028E4
S31508008EE0D7D0012038E04FF48022DEE700F01AFFE1
S31508008EF01F4BD3F8E02591B24FF6FF7399422CD059
S31508008F001C4B03EA82234FF4F030B0FBF3F003FB6B
S31508008F1000F0C0F5F0300221C00AFFF72DFF20BB94
S31508008F20154B00221A80124BD3F8E03599B24FF64A
S31508008F30FF72914214D00F4A02EA83224FF4F033AB
S31508008F40B3FBF2F302FB03F3C3F5F033DB0A0B4A78
S31508008F5013700B4B20221A6038BD4FF48023D2E7DA
S31508008F604FF48022EAE70E20F6E70220F4E700BF76
S31508008F700070FF1F00FCFF03E2040020E00400204D
S31508008F80C000002038B5394BD3F8E02591B24FF62A
S31508008F90FF7399420CD0364B03EA82234FF4F03420
S31508008FA0B4FBF3F403FB04F4C4F5F034E40A4CE030
S31508008FB04FF48023F2E7651CA31CAB4207D80221B5
S31508008FC0204600F09DFE0446F0B1012449E005F56F
S31508008FD08032D202254BD3F8E01588B24FF6FF73DC
S31508008FE098420ED0224B03EA81234FF4F030B0FBAF
S31508008FF0F3F003FB0020FFF791FE042833D1013577
S31508009000DAE74FF48023F0E700F08CFE29E0184AEF
S3150800901002EA83224FF4F033B3FBF2F302FB03F3C5
S31508009020C3F5F033DB0A0433A34219D904F58030BB
S315080090304FF4F033B3FBF2F302FB03F303EBC02068
S31508009040FFF76CFE0428B6D00234084BD3F8E03597
S3150800905099B24FF6FF729142D9D14FF48022D9E7DF
S315080090600524204638BD0524FBE700BF0070FF1F16
S3150800907000FCFF03F8B50646614B1D7805F58032FE
S31508009080D202604BD3F8E01588B24FF6FF739842C8
S315080090904FD05D4B03EA81234FF4F030B0FBF3F079
S315080090A003FB0020FFF73AFE0746564BD3F8E03598
S315080090B099B24FF6FF7291423ED0534A02EA832292
S315080090C04FF4F033B3FBF2F302FB03F3C3F5F032CC
S315080090D0A5EBD224013404F0030404EBD22404F5EE
S315080090E0803003EBC020FFF719FE464BD3F8E03576
S315080090F099B24FF6FF72914221D0434A02EA83227F
S315080091004FF4F033B3FBF2F302FB03F3C3F5F0338A
S31508009110A5EBD322033202F0030202EBD322012E7F
S3150800912010D0022E57D0002E4CD04FF0FF352846CF
S31508009130F8BD4FF48023AFE74FF48022C0E74FF421
S315080091408022DDE7022F19D0012F4DD12F4B1B6846
S31508009150B3F5006FEBD304282DD003212846FFF77B
S315080091600BFE002843D101212046FFF705FE002803
S3150800917040D1264B20221A602546D8E7234B1B6888
S31508009180B3F5006FD3D304280ED003212846FFF782
S31508009190F3FD18BB02212046FFF7EEFD08BB1B4B6B
S315080091A020221A602546C2E7FFF7ECFE0028ECD01D
S315080091B04FF0FF35BBE7FFF7E5FE0028CDD04FF0AF
S315080091C0FF35B4E7022FB2D0012F02D04FF0FF359A
S315080091D0ADE71546ABE780B92546A8E74FF0FF355A
S315080091E0A5E74FF0FF35A2E74FF0FF359FE74FF0B1
S315080091F0FF359CE74FF0FF3599E74FF0FF3596E7C7
S31508009200E00400200070FF1F00FCFF03C0000020E0
S3150800921082B00B4B9A6C42F480529A649B6C03F4AE
S3150800922080530193019B074A48F2050353619368EB
S3150800923023F0180343F00803936002B0704700BF99
S315080092400010024000300240044B9A6842F00102C6
S315080092509A6018601980186880B27047003002401A
S315080092602DE9F04780468A460020FFF703FFB0F154
S31508009270FF3F63D0814600F58035ED02304BD3F8C9
S31508009280E02591B24FF6FF7399420CD02D4B03EAB5
S3150800929082234FF4F032B2FBF3F203FB0255284661
S315080092A0FFF73CFD3EE04FF48023F2E7083C1F2C15
S315080092B016D92B19D3E90067B7F1FF3F08BFB6F1F6
S315080092C0FF3FF3D0B1B24145F0D13846FFF7BCFFB6
S315080092D0B0EB164FEAD1CAF800700020BDE8F08757
S315080092E0174BD3F8E02591B24FF6FF73994220D079
S315080092F0144B03EA82234FF4F035B5FBF3F503FB71
S3150800930005F5C5F5F033A9EBD32909F1030909F0E9
S31508009310030909EBD32909F5803305EBC32528464C
S31508009320FFF7FCFC0238C0B2022805D84FF4FF64E8
S31508009330BDE74FF48023DEE70720CFE70320CDE71C
S315080093400070FF1F00FCFF03431E9BB24FF6FD7221
S31508009350934201D90820704710B582B00C46002305
S31508009360019301A9FFF77CFF019B236002B010BDA2
S31508009370224B1B88B3F5FC7F39D270B506460D46DD
S315080093800120FFF777FEB0F1FF3F32D000F58034B9
S31508009390E4021B4BD3F8E02591B24FF6FF739942CE
S315080093A020D0184B03EA82234FF4F032B2FBF3F2D3
S315080093B003FB024405B9C6B131462846FFF744FF08
S315080093C0114B196846EA00422B46601800F08CFCDF
S315080093D088B90D4A136808331360084A138801339D
S315080093E0138070BD4FF48023DEE72846E8E7122095
S315080093F070470320F5E70220F3E700BFE2040020E8
S315080094000070FF1F00FCFF03C0000020F0B583B00A
S3150800941005460E46002301931746002A4CD1022022
S31508009420FFF728FE0446B0F1FF3F00F031819E4B5E
S3150800943000221A809D4B18709D4B20221A60002F1F
S315080094403CD09C4BD3F8E03599B24FF6FF72914267
S315080094503BD0994A02EA83224FF4F033B3FBF2F386
S3150800946002FB03F3C3F5F032A4EBD224033404F071
S31508009470030404EBD22404F5803003EBC020FFF785
S315080094804DFC022824D0042829D0012F40F004815D
S31508009490032840F00381012F00F0A38031462846B7
S315080094A0FFF766FF002840F0FB807F4B1C88022CE4
S315080094B040F2E180023CCFE00120B1E70121FFF74D
S315080094C05BFC0028BDD00223DFE04FF48022C3E70F
S315080094D004212046FFF750FC002840F0DB80754B3E
S315080094E0D3F8E03599B24FF6FF72914218D0724A16
S315080094F002EA83224FF4F033B3FBF2F302FB03F3E1
S31508009500C3F5F032A4EBD224033404F0030404EBCD
S31508009510D22404F5803003EBC020FFF7FFFB20E0E0
S315080095204FF48022E6E704212046FFF725FCF0B138
S315080095300223AAE04FF480224FF4F033B3FBF2F390
S3150800954002FB03F3C3F5F032A4EBD224033404F090
S31508009550030404EBD22404F5803003EBC020FFF7A4
S31508009560DDFBC31EDBB2012B95D80328DBD0514B9C
S31508009570D3F8E03599B24FF6FF729142DAD04E4AE7
S3150800958002EA8322D8E74C4A02EA81224FF4F031F4
S31508009590B1FBF2F102FB01330344D3E90023B3F133
S315080095A0FF3F08BFB2F1FF3F1DD03F4A1388013382
S315080095B013803F4A1368083313600830B0F5006F0C
S315080095C011D23A4B1B7803F58033DB02394AD2F8BD
S315080095D0E0158CB24FF6FF729442D4D14FF4802234
S315080095E0D4E72020EAE7314B1C7800271EE04FF429
S315080095F080224FF4F033B3FBF2F302FB03F3C3F517
S31508009600F032A4EBD224033404F0030404EBD2248E
S3150800961004F5803003EBC020FFF780FB03287FF4B6
S315080096203DAF214A1388FC3313800137032F3FF6D9
S3150800963035AF204BD3F8E03599B24FF6FF72914219
S31508009640D5D01D4A02EA8322D3E701993046FFF7AF
S315080096508FFE0346C8B90134062C0ED8A542FAD0A7
S31508009660A6B201A93046FFF7FBFD03460028ECD059
S315080096700728F0D009E00124EEE702210B4B187801
S31508009680FFF77AFB70B94FF48073184603B0F0BD44
S315080096900423FAE70223F8E70A23F6E70A23F4E79E
S315080096A00223F2E70223F0E7E2040020E0040020A8
S315080096B0C00000200070FF1F00FCFF032DE9F047E3
S315080096C0054600F043FB002840F0DD820446FFF71C
S315080096D09FFDBE4B01221A70BD4BD3F8E02591B20F
S315080096E04FF6FF7399420CD0BA4B03EA82234FF424
S315080096F0F037B7FBF3F703FB07F7C7F5F037FF0AB1
S315080097000CE04FF48023F2E71A18B3490A6092ED89
S31508009710007B0833B3F5006FF6D30137AC4BD3F8AB
S31508009720E02591B24FF6FF7399421AD0A94B03EA86
S3150800973082234FF4F036B6FBF3F603FB06F6C6F5BE
S31508009740F036F60A321DBA420ED907F580324FF4C2
S31508009750F030B0FBF3F003FB00F000EBC22000236F
S31508009760D8E74FF48023E4E74FF00008974B83F8D7
S315080097700080C2464746C14602E008F101080136A4
S31508009780934BD3F8E03599B24FF6FF72914228D041
S31508009790904A02EA83224FF4F033B3FBF2F302FB5A
S315080097A003F3C3F5F033DB0A191DB1421CD906F5DC
S315080097B080304FF4F033B3FBF2F302FB03F303EB11
S315080097C0C020FFF7ABFA431EDBB2012BD5D903281D
S315080097D0D5D1B9F1000F00D1B24609F101093746D2
S315080097E0CDE74FF48022D6E7B8F1000F16D1B9F1CC
S315080097F0000F4CD0AAEB0301033101F003010B441F
S3150800980003F580334FF4F030B0FBF2F002FB00F0C2
S3150800981000EBC320FFF782FA042814D06C4BD3F868
S31508009820E02591B24FF6FF73994235D0694B03EAAA
S3150800983082234FF4F036B6FBF3F603FB06F6C6F5BD
S31508009840F036F60A42E0624BD3F8E03599B24FF6A5
S31508009850FF72914218D05F4A02EA83224FF4F0332E
S31508009860B3FBF2F302FB03F3C3F5F033A7EBD32004
S31508009870013000F00300012100EBD320FFF77CFA4A
S315080098800028CBD00224FFE14FF48022E6E700202F
S31508009890FFF7D0FA0446F7E14FF48023C9E74FF4FF
S315080098A0802143E0B31A013303F00303134403F59D
S315080098B080334FF4F030B0FBF1F001FB00F000EB21
S315080098C0C320FFF72BFA002852D00136404BD3F8B5
S315080098D0E03599B24FF6FF72914257D03D4A02EAF7
S315080098E083224FF4F033B3FBF2F302FB03F3C3F521
S315080098F0F033DB0A0433B3424BD906F580304FF414
S31508009900F033B3FBF2F302FB03F303EBC020FFF7DC
S3150800991005FA0128D9D12E4BD3F8E03599B24FF67E
S31508009920FF729142BBD02B4901EA83214FF4F033F1
S31508009930B3FBF1F301FB03F3C3F5F033DA0AB6EB35
S31508009940D32FAFD0931CB342ACD0B31A033303F072
S315080099500303134403F580334FF4F030B0FBF1F002
S3150800996001FB00F000EBC320FFF7D8F90328ACD1C0
S315080099701A4B1E70012200210846FFF747FDB0F575
S31508009980807F40F084814FF0010904E04FF4802283
S31508009990A7E74FF000090E4BD3F8E02591B24FF632
S315080099A0FF7399420ED00B4B03EA82234FF4F0362D
S315080099B0B6FBF3F603FB06F6C6F5F036F60A4FF0E5
S315080099C0000842E04FF48023F0E700BFD8040020E7
S315080099D00070FF1F00FCFF03DC040020E0040020E9
S315080099E0AF4BD3F8E03599B24FF6FF72914255D096
S315080099F0AC4A02EA83224FF4F033B3FBF2F302FBDC
S31508009A0003F3C3F5F033D90AB6EBD32F02D08B1C78
S31508009A10B34246D1731A013303F003030B4403F52B
S31508009A2080334FF4F030B0FBF2F002FB00F000EBAD
S31508009A30C320FFF773F938B9B8F1000F40F0298150
S31508009A40994B1E7008F101080136954BD3F8E0359D
S31508009A5099B24FF6FF72914237D0924A02EA8322B0
S31508009A604FF4F033B3FBF2F302FB03F3C3F5F03321
S31508009A70DB0A191DB1422BD906F580304FF4F033B5
S31508009A80B3FBF2F302FB03F303EBC020FFF746F93F
S31508009A900228A5D00328D7D13746D5E74FF4802228
S31508009AA0A9E7731A033303F003030B4403F5803362
S31508009AB04FF4F030B0FBF2F002FB00F000EBC320ED
S31508009AC0FFF72CF90328BFD1B6E74FF48022C7E782
S31508009AD0B8F1000F06D0754B00221A802022744B6D
S31508009AE01A602AE0DBB2FA1AD2B2013202F0030295
S31508009AF01344D8B26C4B18700221FFF73DF90028C1
S31508009B00E9D00224C0E04FF480214FF4F030B0FBD6
S31508009B10F1F001FB00331344D3E90001B1F1FF3F33
S31508009B2008BFB0F1FF3F1CD060490B8801330B809A
S31508009B305F490B6808330B600832B2F5006F10D224
S31508009B40594B1B7803F58033DB025549D1F8E005FC
S31508009B5086B24FF6FF718E42D5D0524901EA80216E
S31508009B60D3E7514B1F7827E04FF480224FF4F033A8
S31508009B70B3FBF2F302FB03F3C3F5F033DE0AB7EBEC
S31508009B80D32F25D0B31CBB4222D0BF1B033707F007
S31508009B900307374407F580304FF4F033B3FBF2F38D
S31508009BA002FB03F303EBC020FFF7B8F8032872D1D2
S31508009BB03E4A1388FC331380394BD3F8E03599B203
S31508009BC04FF6FF729142CFD0364A02EA8322CDE79A
S31508009BD0354B1B789B1B013303F003031E4406F524
S31508009BE080314FF4F033B3FBF2F302FB03F303EBDC
S31508009BF0C12023E04FF40061FFF777F8102829D039
S31508009C00274BD3F8E03599B24FF6FF72914229D027
S31508009C10244A02EA83224FF4F033B3FBF2F302FB41
S31508009C2003F3C3F5F032A6EBD226013606F0030697
S31508009C3006EBD22606F5803203EBC220B74214D0D3
S31508009C40002DD7D10121304600F05AF80028D7D088
S31508009C50012419E00121304600F052F80028CFD03F
S31508009C60012411E04FF48022D5E700F05BF8B9F142
S31508009C70000F09D100210846FFF77AFB68B11228C0
S31508009C8002D0022400E00E242046BDE8F0870C240A
S31508009C90FAE70A24F8E70A24F6E70446F4E700BFD9
S31508009CA00070FF1F00FCFF03E0040020E204002010
S31508009CB0C000002038B504460D46FFF759FB1228A8
S31508009CC000D038BD002229462046FFF79FFBF8E75B
S31508009CD008B5431E9BB24FF6FD72934201D9082080
S31508009CE008BDFFF7E7FFFBE710B5014603484CF24E
S31508009CF0FB3404610020FDF7FBF910BD002002408B
S31508009D0000B587B0002301930293059104900123BF
S31508009D10039301A902A8FDF799FA00B1012007B03B
S31508009D205DF804FB084B1A6822F480621A601A6808
S31508009D3042F480521A601A6822F480521A601A682D
S31508009D4042F480621A607047002002400020704783
S31508009D5008B502F044FB10B102684068904708BD98
S31508009D60EFF305832BB9064B186828B901221A6048
S31508009D7070476FF0050070474FF0FF30704700BF1F
S31508009D80340C0020EFF3058373B90A4B1B68012BCB
S31508009D900DD110B50024084BDC77064B02221A6059
S31508009DA001F0F0FB204610BD6FF0050070474FF03C
S31508009DB0FF307047340C002000ED00E008B5EFF3E3
S31508009DC0058343B901F068FF40B1022808D101F0C4
S31508009DD02FFC002006E06FF0050003E0012001E0FB
S31508009DE04FF0FF3008BDF0B587B000240594EFF3B7
S31508009DF0058474BB68B322B31568936903B918233D
S31508009E005C1E372C49D8546814F0010F47D156699F
S31508009E106EB14FEA960C94682CB1D768A72F02D971
S31508009E20176907B1C6B92CB14FF0FF340EE04FF0F1
S31508009E30800CF0E7D4688CB9146994B14FF0FF34FC
S31508009E4004E01546002418234FF0800C012C0AD094
S31508009E50ACB1059807B0F0BD0124F7E74FF0FF3421
S31508009E60F4E70024F2E714699268029201940093D9
S31508009E700B466246294601F017FB0590E9E705AA55
S31508009E80019200930B461FFA8CF2294601F047FB14
S31508009E900128DED000230593DBE70020DAE700205F
S31508009EA0D8E708B5EFF3058323B930B101F04EFDC5
S31508009EB0002008BD6FF00500FBE76FF00300F8E728
S31508009EC008B5EFF3058333B908B9002008BD01F0DA
S31508009ED0C5FC0020FAE76FF00500F7E72DE9F04327
S31508009EE083B0EFF30587002F43D10646894615460A
S31508009EF01C4600283FD0082002F0BCFC80460028FB
S31508009F003BD006604560B9F1000F00D0012704B3C5
S31508009F102068A36813B1E2682B2A10D853B14FF012
S31508009F20FF33DBB10024404602F026FD204603B08D
S31508009F30BDE8F083E3687BB14FF0FF33F1E70193A7
S31508009F400F4B009343463A46012102F093F8044624
S31508009F500CE020460023E4E70023E2E7084B0093E1
S31508009F6043463A46012102F069F80446002CDDD141
S31508009F70D9E70024DAE70024D8E70446D6E700BF85
S31508009F80519D0008EFF305836BB90A4670B100B519
S31508009F9083B00093042102F097F8012809D1002024
S31508009FA003B05DF804FB6FF0050070476FF003001F
S31508009FB070476FF00200F3E708B5EFF30583CBB9F6
S31508009FC0A0B1836813B1C2681F2A0BD82BB14FF012
S31508009FD0FF338BB900F050FA08BDC36843B14FF0A0
S31508009FE0FF33F6E7184600F022FAF5E70023F0E714
S31508009FF00023EEE70020EFE70020EDE7F8B110B503
S3150800A00082B00C46B1F1807F1CD2EFF305829AB17B
S3150800A0100022019201AA00F04DFBB8B1019BC3B121
S3150800A0204FF0E0234FF08052C3F8042DBFF34F8F53
S3150800A030BFF36F8F204607E000F0F0FA04E06FF0F8
S3150800A040030070476FF0030002B010BD6FF0020006
S3150800A050FAE72046F8E770B5B0B10C460646B1F106
S3150800A060807F14D2EFF3058353B100F0C9FA054691
S3150800A0702146304600F0BAFA58B96FF0020508E0F2
S3150800A08000F08DFA054604E06FF0030501E06FF075
S3150800A0900305284670BD40B370B582B00C461D4610
S3150800A0A08446B1F1807F23D2EFF3058323BB12F0F8
S3150800A0B0010610D0012312F0020F0ED000220095DF
S3150800A0C02146604600F0E6F94EB1844312D0B5B198
S3150800A0D06FF001000EE00023EDE70122EFE70442EE
S3150800A0E008D17DB16FF0010004E06FF003007047FE
S3150800A0F06FF0030002B070BD6FF00500FAE76FF06D
S3150800A1000200F7E76FF00200F4E770B5EFF3058396
S3150800A110002B3CD1044600B1436813F0010600D079
S3150800A120012613F0080F35D144B3A16811B1E368CD
S3150800A1304F2B18D891B14FF0FF336BBB16B30420E1
S3150800A14000F040FD05461DB304B1246821462846A3
S3150800A15000F0D2FFE6B145F0010519E0E3687BB1EE
S3150800A1604FF0FF33E9E726B1042000F036FD054637
S3150800A170E9E7012000F031FD0546E4E70023DCE7C6
S3150800A1800023DAE7012000F01DFD0546DBE7002580
S3150800A190284670BD0025FBE70025F9E7EFF30582A1
S3150800A1A0DAB910B503460C4620F0010003F00101A8
S3150800A1B0012B15D941B1214600F027FF012812D0FD
S3150800A1C09CB16FF001000FE0214600F04BFE01281C
S3150800A1D00ED07CB16FF0010006E06FF00500704705
S3150800A1E06FF0030000E0002010BD6FF00200FBE7EF
S3150800A1F00020F9E76FF00200F6E7EFF30582BAB937
S3150800A20008B5034620F0010003F00101012B12D91D
S3150800A21029B100F0F1FC012810D1002008BD002367
S3150800A2201A46194600F0FEFB01280AD10020F5E778
S3150800A2306FF0050070476FF00300EFE76FF002005C
S3150800A240ECE76FF00200E9E770B582B0EFF305833B
S3150800A250002B3AD1144600283BD000293BD06AB3DC
S3150800A26093684BB1D2684F2A06D9226922B101FBFD
S3150800A27000F56669AE421BD273B14FF0FF3363BB7C
S3150800A280002200F0ABFB054605B304B1246821465D
S3150800A290284600F031FF19E0E3688BB9236913B14A
S3150800A2A04FF0FF33EBE763696BB14FF0FF33E6E737
S3150800A2B00025009500F048FB0546E5E70023DEE7A4
S3150800A2C04FF0FF33DBE70023D9E70025284602B025
S3150800A2D070BD0025FAE70025F8E70025F6E710B572
S3150800A2E082B01C46EFF30583C3B118B329B33CBB50
S3150800A2F00023019301AA00F09FFC012823D10198AD
S3150800A30050B14FF0E0234FF08052C3F8042DBFF34D
S3150800A3104F8FBFF36F8F002002B010BDB0B1C1B12F
S3150800A3200023224600F07EFB012815D0B4B16FF059
S3150800A3300100F1E76FF00300EEE76FF00300EBE7CB
S3150800A3406FF00300E8E76FF00200E5E76FF003003F
S3150800A350E2E76FF00300DFE70020DDE76FF00200B9
S3150800A360DAE710B582B01C46EFF30583C3B110B324
S3150800A37021B334BB0023019301AA00F066FE01282D
S3150800A38022D1019850B14FF0E0234FF08052C3F824
S3150800A390042DBFF34F8FBFF36F8F002002B010BD9F
S3150800A3A0A8B1B9B1224600F0AEFC012815D0B4B167
S3150800A3B06FF00100F2E76FF00300EFE76FF00300BC
S3150800A3C0ECE76FF00300E9E76FF00200E6E76FF0ED
S3150800A3D00300E3E76FF00300E0E70020DEE76FF035
S3150800A3E00200DBE7034B0360034B0B60802313601B
S3150800A3F0704700BF8C0B00208C090020034B0360BC
S3150800A400034B0B604FF4807313607047E408002019
S3150800A410E40400201AB9084205D110467047814362
S3150800A42003D000207047012070470120704780B193
S3150800A43010B582B0044620230193019B202B11D02E
S3150800A4404FF0500383F31188BFF36F8FBFF34F8F1D
S3150800A450FEE74FF0500383F31188BFF36F8FBFF306
S3150800A4604F8FFEE7002340F8043B00F02DF9012347
S3150800A4702377204602B010BD38B5202002F0FAF93D
S3150800A480044628B1002540F8045B00F01DF925773D
S3150800A490204638BD88B12DE9F0410C4616461D46C2
S3150800A4A00746B1F1807F11D34FF0500383F311882B
S3150800A4B0BFF36F8FBFF34F8FFEE74FF0500383F361
S3150800A4C01188BFF36F8FBFF34F8FFEE741B94FF087
S3150800A4D0500383F31188BFF36F8FBFF34F8FFEE7E7
S3150800A4E001F0DAFB50B9069B43B14FF0500383F3F2
S3150800A4F01188BFF36F8FBFF34F8FFEE701F098F80F
S3150800A500D7F800802A4621464046FFF783FFF8B170
S3150800A5108EB328EA04033B600023069301F022F970
S3150800A520069B93B148B94FF0E0234FF08052C3F829
S3150800A530042DBFF34F8FBFF36F8F01F0A1FC804648
S3150800A54010F0007F1AD028F07F484046BDE8F08119
S3150800A550069B002BE2D05EB900210DB141F0806167
S3150800A560069A2143381D01F06BFA4FF00008D5E72B
S3150800A5704FF08071F1E700230693CFE701F0C2FFA1
S3150800A580D7F800802A4621464046FFF743FF18B110
S3150800A59016B128EA04043C6001F0D6FFD3E770B18F
S3150800A5A070B50C460546B1F1807F11D34FF05003C4
S3150800A5B083F31188BFF36F8FBFF34F8FFEE74FF01A
S3150800A5C0500383F31188BFF36F8FBFF34F8FFEE7F6
S3150800A5D001F098FF2E6826EA04042C6001F0B4FF07
S3150800A5E0304670BD08B5FFF7DAFF08BD08B50A465C
S3150800A5F000230146014801F005FF08BDE5A500084E
S3150800A600EFF311834FF0500282F31188BFF36F8F77
S3150800A610BFF34F8F006883F311887047F8B568B1A8
S3150800A6200D460446B1F1807F11D34FF0500383F3F2
S3150800A6301188BFF36F8FBFF34F8FFEE74FF05003BC
S3150800A64083F31188BFF36F8FBFF34F8FFEE700F1D7
S3150800A6500C0600F0EDFF206923682B4323600027D2
S3150800A6600AE0216832EA010105D111E0216841F0CA
S3150800A670007101F073FA2846B0420ED045680368A7
S3150800A68023F07F4213F0806FEBD121681142F2D09C
S3150800A69013F0807FEAD01743E8E7236823EA070325
S3150800A6A0236001F05FF82068F8BD08B5FFF7B6FF2C
S3150800A6B008BD000008B513460A460146014801F0E0
S3150800A6C0A1FE08BDABA6000800F1080343604FF0E1
S3150800A6D0FF328260C3600361002303607047002372
S3150800A6E00361704743684B609A688A605160996055
S3150800A6F00861036801330360704730B40D68B5F12B
S3150800A700FF3F11D000F108031C465B681A68AA428D
S3150800A710FAD963684B6099608C6061600861036868
S3150800A7200133036030BC70470469F2E70369416886
S3150800A73082688A60416851605A68824206D000225F
S3150800A74002611A68013A1A601868704782685A6086
S3150800A750F5E70346406A18B11B6B1868C0F1380064
S3150800A760704710B5044601F0CDFEA26BE36B9A4222
S3150800A77004D0002401F0E8FE204610BD0124F9E7C4
S3150800A78010B5044601F0BEFEA36B23B9012401F0FF
S3150800A790DBFE204610BD0024F9E770B504461546D1
S3150800A7A0866B026C5AB903681BB100200136A66392
S3150800A7B070BD806801F0CCFA0023A360F6E76DB996
S3150800A7C0406802F0C5F96368226C13446360A268A6
S3150800A7D0934219D3236863602846E7E7C06802F006
S3150800A7E0B7F9E368226C51429B1AE36022689342E8
S3150800A7F002D2A3680B44E360022D01D00020D5E7FE
S3150800A80026B1013E0020D1E72846CFE70020CDE754
S3150800A8100346026C6AB110B50846D9681144D96076
S3150800A8209C68A14201D31968D960D96802F090F9E9
S3150800A83010BD704738B5054601F064FE95F84540E9
S3150800A84064B201E0013C64B2002C0ADD6B6A43B1D4
S3150800A85005F1240001F03CF90028F3D001F010FAC4
S3150800A860F0E7FF2385F8453001F06EFE01F04AFE59
S3150800A87095F8444064B201E0013C64B2002C0ADD5C
S3150800A8802B6943B105F1100001F022F90028F3D035
S3150800A89001F0F6F9F0E7FF2385F8443001F054FE9D
S3150800A8A038BD38B5E0B10D46044601F02BFE2368E5
S3150800A8B0E26B216C01FB0230A0600020A06363609C
S3150800A8C0013A02FB0133E360FF2384F8443084F83D
S3150800A8D04530FDB9236963B901F036FE012038BD5C
S3150800A8E04FF0500383F31188BFF36F8FBFF34F8F79
S3150800A8F0FEE704F1100001F0EBF80028ECD04FF069
S3150800A900E0234FF08052C3F8042DBFF34F8FBFF3F7
S3150800A9106F8FE1E704F11000FFF7D6FE04F124007B
S3150800A920FFF7D2FED8E738B51D46049C0B4649B951
S3150800A9302460E063236401212046FFF7B2FF84F810
S3150800A9404C5038BD2260F4E740B94FF0500383F30A
S3150800A9501188BFF36F8FBFF34F8FFEE710B584B032
S3150800A9601C46844653B192B189B94FF0500383F31C
S3150800A9701188BFF36F8FBFF34F8FFEE74FF0500379
S3150800A98083F31188BFF36F8FBFF34F8FFEE76AB16A
S3150800A99050230393039B502B13D04FF0500383F39C
S3150800A9A01188BFF36F8FBFF34F8FFEE70029EFD0F3
S3150800A9B04FF0500383F31188BFF36F8FBFF34F8FA8
S3150800A9C0FEE7039B012384F8463000949DF818306F
S3150800A9D06046FFF7A8FF204604B010BD40B94FF007
S3150800A9E0500383F31188BFF36F8FBFF34F8FFEE7D2
S3150800A9F0F0B583B00D461446064601FB00F050300C
S3150800AA0001F038FF074650B1002380F84630009021
S3150800AA10234600F1500229463046FFF784FF3846A0
S3150800AA2003B0F0BDF0B585B0019288B10F461D465A
S3150800AA300446B1B1022D20D1E36B012B1DD04FF096
S3150800AA40500383F31188BFF36F8FBFF34F8FFEE771
S3150800AA504FF0500383F31188BFF36F8FBFF34F8F07
S3150800AA60FEE7036C002BE5D04FF0500383F3118803
S3150800AA70BFF36F8FBFF34F8FFEE701F00DF9064660
S3150800AA8058B9019B002B48D04FF0500383F3118827
S3150800AA90BFF36F8FBFF34F8FFEE700263DE02A46D0
S3150800AAA039462046FFF779FE636A7BB948B14FF00D
S3150800AAB0E0234FF08052C3F8042DBFF34F8FBFF346
S3150800AAC06F8F01F041FD012005B0F0BD04F12400AF
S3150800AAD000F0FEFF0028F4D04FF0E0234FF080523C
S3150800AAE0C3F8042DBFF34F8FBFF36F8FE9E701F06B
S3150800AAF02BFD0020E8E702A801F074F8012619E00A
S3150800AB00002384F8443021E0002384F8453023E00C
S3150800AB102046FFF78FFE00F025FE01F0F3FCA26B3E
S3150800AB20E36B9A42BBD3022DB9D0019B002BDED032
S3150800AB30002EE0D001F008FD00F07AFD01F0E2FCFD
S3150800AB4094F8442052B2B2F1FF3FD9D094F8452088
S3150800AB5052B2B2F1FF3FD7D001F0F6FC01A902A824
S3150800AB6001F04CF8D8B92046FFF7FBFD0028CFD0F6
S3150800AB70019904F1100000F04BFF2046FFF75AFE3A
S3150800AB8000F0F0FD0028C8D14FF0E0234FF08052C6
S3150800AB90C3F8042DBFF34F8FBFF36F8FBDE7204671
S3150800ABA0FFF748FE00F0DEFD00208DE748B108B546
S3150800ABB0002181600160C1600B460A46FFF732FF3B
S3150800ABC008BD704710B5024600210120FFF706FFB1
S3150800ABD00446FFF7EBFF204610BD10B582B00B46C2
S3150800ABE00090002211460120FFF7AEFE0446FFF74B
S3150800ABF0DDFF204602B010BD38B538B10446856879
S3150800AC0001F044F885420AD0002038BD4FF05003C1
S3150800AC1083F31188BFF36F8FBFF34F8FFEE7E368A7
S3150800AC20013BE3600BB10120EFE71A4619462046BF
S3150800AC30FFF7F8FE0120E8E72DE9F84390B10F4643
S3150800AC4016461C460546B1B1022C20D1EB6B012BEA
S3150800AC501DD04FF0500383F31188BFF36F8FBFF3F6
S3150800AC604F8FFEE74FF0500383F31188BFF36F8FC2
S3150800AC70BFF34F8FFEE7036C002BE5D04FF0500370
S3150800AC8083F31188BFF36F8FBFF34F8FFEE701F091
S3150800AC905FFDEFF311884FF0500383F31188BFF37C
S3150800ACA06F8FBFF34F8FAA6BEB6B9A4206D3022CBA
S3150800ACB004D0002088F31188BDE8F88395F84590FC
S3150800ACC04FFA89F9AB6B224639462846FFF765FDE8
S3150800ACD0B9F1FF3F06D009F101035BB285F84530AB
S3150800ACE00120E7E76B6A0BB90120E3E705F12400C9
S3150800ACF000F0EEFE18B126B101203060DAE7012037
S3150800AD00D8E70120D6E7F0B585B0019290B10F4695
S3150800AD100446C1B100F0C0FF064600BB019B002BEC
S3150800AD205ED04FF0500383F31188BFF36F8FBFF3E4
S3150800AD304F8FFEE74FF0500383F31188BFF36F8FF1
S3150800AD40BFF34F8FFEE7036C002BE3D04FF05003A1
S3150800AD5083F31188BFF36F8FBFF34F8FFEE700268B
S3150800AD603EE039462046FFF753FD013DA5632369BA
S3150800AD7023B901F0E9FB012005B0F0BD04F110008C
S3150800AD8000F0A6FE0028F4D04FF0E0234FF08052E2
S3150800AD90C3F8042DBFF34F8FBFF36F8FE9E701F0B8
S3150800ADA0D3FB0020E8E702A800F01CFF012621E0FB
S3150800ADB0002384F8443029E0002384F845302BE04A
S3150800ADC02046FFF737FD00F0CDFC09E02046FFF7E7
S3150800ADD031FD00F0C7FC2046FFF7D2FC00283FD122
S3150800ADE001F090FBA56B002DBBD1019B002BD6D0A3
S3150800ADF0002ED8D001F0A8FB00F01AFC01F082FB67
S3150800AE0094F844305BB2B3F1FF3FD1D094F84530A3
S3150800AE105BB2B3F1FF3FCFD001F096FB01A902A8C0
S3150800AE2000F0ECFE0028D1D12046FFF7A9FC002847
S3150800AE30C6D0019904F1240000F0EAFD2046FFF788
S3150800AE40F9FC00F08FFC0028CAD14FF0E0234FF040
S3150800AE508052C3F8042DBFF34F8FBFF36F8FBFE740
S3150800AE60002089E770B584B0019158B10446036C97
S3150800AE708BB14FF0500383F31188BFF36F8FBFF385
S3150800AE804F8FFEE74FF0500383F31188BFF36F8FA0
S3150800AE90BFF34F8FFEE700F0FFFE054650B9019B52
S3150800AEA05BB14FF0500383F31188BFF36F8FBFF385
S3150800AEB04F8FFEE70026354655E0064653E0013B30
S3150800AEC0A36323683BB123694BB901F03DFB012617
S3150800AED0304604B070BD00F0DFFFA060F3E704F170
S3150800AEE0100000F0F5FD0028EFD04FF0E0234FF0FA
S3150800AEF08052C3F8042DBFF34F8FBFF36F8FE4E77B
S3150800AF0046B14FF0500383F31188BFF36F8FBFF339
S3150800AF104F8FFEE701F018FBDAE702A800F062FEA1
S3150800AF2001252AE0002384F8443032E0002384F81F
S3150800AF30453034E001F0E6FAA06800F0BDFE0646AA
S3150800AF4001F002FB3BE02046FFF774FC00F00AFC28
S3150800AF5009E02046FFF76EFC00F004FC2046FFF7E8
S3150800AF600FFC002842D101F0CDFAA36B002BA6D125
S3150800AF70019B002BC4D0002DCFD001F0E5FA00F0DC
S3150800AF8057FB01F0BFFA94F844305BB2B3F1FF3FC8
S3150800AF90C8D094F845305BB2B3F1FF3FC6D001F094
S3150800AFA0D3FA01A902A800F029FE0028D1D120462B
S3150800AFB0FFF7E6FB0028C6D02368002BBAD0019914
S3150800AFC004F1240000F024FD2046FFF733FC00F0CE
S3150800AFD0C9FB0028C7D14FF0E0234FF08052C3F8D1
S3150800AFE0042DBFF34F8FBFF36F8FBCE70EB9002652
S3150800AFF06EE701F087FA2046FFF7ABFB0146A0682B
S3150800B00000F0EEFE01F0A0FAF1E780B170B50C464B
S3150800B0100546866800F03AFE864211D02146284643
S3150800B020FFF720FF80B1EB680133EB600CE04FF0CF
S3150800B030500383F31188BFF36F8FBFF34F8FFEE77B
S3150800B040EB680133EB60012070BD2DE9F843B0B120
S3150800B0500D4690460446D9B101F07AFBEFF3118705
S3150800B0604FF0500383F31188BFF36F8FBFF34F8FF1
S3150800B070A66BCEB9002087F31188BDE8F8834FF098
S3150800B080500383F31188BFF36F8FBFF34F8FFEE72B
S3150800B090036C002BE0D04FF0500383F31188BFF305
S3150800B0A06F8FBFF34F8FFEE794F844904FFA89F9F4
S3150800B0B029462046FFF7ACFB731EA363B9F1FF3F91
S3150800B0C006D009F101035BB284F844300120D2E7C7
S3150800B0D023690BB90120CEE704F1100000F0F8FC53
S3150800B0E030B1B8F1000F05D00120C8F80000C2E75A
S3150800B0F00120C0E70120BEE70023072B0CD8074A2A
S3150800B10052F833200AB10133F7E7044A42F83310FC
S3150800B11002EBC30250607047704700BF380C00202E
S3150800B12070B504460D46164601F0ECF994F844301D
S3150800B1305BB2B3F1FF3F0DD094F845305BB2B3F183
S3150800B140FF3F0BD001F000FAA36B5BB12046FFF777
S3150800B15071FB70BD002384F84430EDE7002384F8C2
S3150800B1604530EFE73246294604F1240000F094FC06
S3150800B170ECE70000084B1B681B6823B9074B4FF028
S3150800B180FF321A607047044B1B68DB68DB685A6835
S3150800B190024B1A60704700BFE80C0020800C0020A4
S3150800B1A02DE9F04780460D4617469946089EDDF874
S3150800B1B024A00A9C9200A521206B01F044FC236B75
S3150800B1C007F18042013A03EB820727F00707002DB3
S3150800B1D042D04FF0000CBCF10F0F09D815F80C300F
S3150800B1E004EB0C0282F8343013B10CF1010CF2E7CF
S3150800B1F0002384F84330372E00D93726E662E66402
S3150800B20000252565201DFFF76AFA04F11800FFF7E7
S3150800B21066FA2461C6F13806A6616462C4F8A050CD
S3150800B22084F8A4504C22294604F1540001F00BFC82
S3150800B2300B4BA36503F16802E265D03323664A46E1
S3150800B2404146384601F030F92060BAF1000F01D0C6
S3150800B250CAF80040BDE8F087002384F83430CAE70E
S3150800B260CC92002038B5002407E004EB8402930052
S3150800B2700E481844FFF728FA0134372CF5D90C4D37
S3150800B2802846FFF721FA0B4C2046FFF71DFA0A4815
S3150800B290FFF71AFA0948FFF717FA0948FFF714FAE9
S3150800B2A0084B1D60084B1C6038BD00BF140D0020FC
S3150800B2B0000D0020EC0C0020D00C0020BC0C002057
S3150800B2C0A40C0020E80C0020E40C002010B504466D
S3150800B2D001F018F9224A136801331360214B1B68E1
S3150800B2E05BB1214B1B686BB91E4B1B68DA6AE36AB4
S3150800B2F09A4207D81B4B1C6004E01A4B1C60136863
S3150800B300012B29D0194A1368013313606364E06A74
S3150800B310174B1B68984201D9154B186000EB800043
S3150800B320211D144B03EB8000FFF7DCF901F00CF943
S3150800B3300D4B1B687BB10B4B1B68DA6AE36A9A42B2
S3150800B34009D24FF0E0234FF08052C3F8042DBFF323
S3150800B3504F8FBFF36F8F10BDFFF784FFD2E700BF93
S3150800B360A00C002074110020940C0020840C0020EE
S3150800B370980C0020140D002010B50446543001F036
S3150800B3806BFB94F8A53063B1012B11D0022B0ED0BC
S3150800B3904FF0500383F31188BFF36F8FBFF34F8FBE
S3150800B3A0FEE7206B01F0E8FA204601F0E5FA10BD49
S3150800B3B0204601F0E1FAFAE70F4B1B68D3B110B546
S3150800B3C001F0A0F80D4BDB68DC68201DFFF7AEF92D
S3150800B3D00B4A1368013B1360074A1368013B136065
S3150800B3E001F0B2F82046FFF7C7FF034B1B68002B96
S3150800B3F0E6D110BD704700BFB80C0020BC0C002079
S3150800B400A00C002008B5FFF7D7FF074B1B68012BD8
S3150800B410F9D94FF0E0234FF08052C3F8042DBFF35B
S3150800B4204F8FBFF36F8FEEE7140D002070B50446FB
S3150800B4300D46174B1E68174B18680430FFF776F948
S3150800B440B4F1FF3F0DD03444124B1B685C60A64232
S3150800B45010D9114B18680F4B19680431FFF74DF9CD
S3150800B46070BD002DEFD00B4B196804310B48FFF760
S3150800B47039F9F5E70A4B1868064B19680431FFF7DE
S3150800B4803CF9084B1B68A342EAD9064B1C60E7E760
S3150800B4909C0C002074110020E40C0020A40C002051
S3150800B4A0E80C0020800C002030B587B00B9C7CB1DE
S3150800B4B00C9DB5B1A8250495049DA82D1AD04FF06A
S3150800B4C0500383F31188BFF36F8FBFF34F8FFEE7E7
S3150800B4D04FF0500383F31188BFF36F8FBFF34F8F7D
S3150800B4E0FEE74FF0500383F31188BFF36F8FBFF366
S3150800B4F04F8FFEE7049D0C9D2C63022485F8A5401A
S3150800B50000240394029505AC01940A9C0094FFF765
S3150800B51047FE0C98FFF7DAFE059807B030BD2DE90F
S3150800B520F04385B00746884614461E46900001F04B
S3150800B530A1F908B38146A82001F09CF90546A8B1EF
S3150800B540C0F83090002380F8A530039302900D9B35
S3150800B55001930C9B00933346224641463846FFF733
S3150800B5601FFE2846FFF7B2FE012007E0484601F015
S3150800B57003FA4FF0FF3001E04FF0FF3005B0BDE8A9
S3150800B580F083000010B588B000240594069407AA35
S3150800B59006A905A8FEF726FF059B0293069B0193BD
S3150800B5A000942346079A1A491A48FFF77DFF1A4B53
S3150800B5B01860E8B100F010FD01281AD14FF05003C9
S3150800B5C083F31188BFF36F8FBFF34F8F134B1B683D
S3150800B5D05433134A1360134B4FF0FF321A60124B61
S3150800B5E001221A60114B00221A6001F025F803E0C7
S3150800B5F00020B0F1FF3F01D008B010BD4FF0500356
S3150800B60083F31188BFF36F8FBFF34F8FFEE700BF39
S3150800B6105CD2000805B400087C0C002074110020D8
S3150800B620C8000020800C0020940C00209C0C0020F0
S3150800B630024A136801331360704700BF780C002074
S3150800B640014B1868704700BF9C0C0020F8B53A4BB0
S3150800B6501B68002B69D1394B1D6801351D60C5B9BA
S3150800B660374B1B681B6843B14FF0500383F31188AF
S3150800B670BFF36F8FBFF34F8FFEE7314A1168314B27
S3150800B680186810601960304A136801331360FFF7B1
S3150800B69071FD2E4B1B68AB423DD900272C4B1B680E
S3150800B6A0DB6A03EB83039A002A4B9B58012B00D9CC
S3150800B6B00127294B1B68002B3CD001273AE00127BC
S3150800B6C01F4B1B681B6843B31D4B1B68DB68DC6894
S3150800B6D063689D4226D3261D3046FFF727F8A36ADE
S3150800B6E01BB104F11800FFF721F8E36A1B4A126838
S3150800B6F0934201D9194A136003EB83039A00314632
S3150800B70014481044FEF7EEFFE26A114B1B68DB6A29
S3150800B7109A42D4D2D4E70027D2E70C4B4FF0FF3237
S3150800B7201A60BBE7094A1360B8E70D4A1368013384
S3150800B730136000273846F8BD780C00209C0C0020C2
S3150800B740E80C0020E40C0020880C0020800C002067
S3150800B75074110020140D00208C0C0020980C002079
S3150800B760900C002038B5354B1B6843B94FF0500391
S3150800B77083F31188BFF36F8FBFF34F8FFEE700F097
S3150800B780C1FE2E4B1A68013A1A601B68002B4FD16E
S3150800B7902B4B1B680BB900244BE00024294B1B6874
S3150800B7A01BB3284BDB68DC6804F11800FEF7BEFF04
S3150800B7B0251D2846FEF7BAFFE06A234B1B68984208
S3150800B7C001D9214B186000EB800029461F4B03EB7B
S3150800B7D08000FEF787FFE26A1D4B1B68DB6A9A4208
S3150800B7E0DCD31C4B01221A60D8E70CB1FFF7C2FC68
S3150800B7F0194B1C6884B9174B1C68D4B14FF0E02369
S3150800B8004FF08052C3F8042DBFF34F8FBFF36F8FED
S3150800B81001240EE0013C07D0FFF718FF0028F9D0F5
S3150800B8200C4B01221A60F5E70B4B00221A60E2E77F
S3150800B830002400F089FE204638BD00BF780C0020A1
S3150800B840A00C0020D00C0020980C0020140D00201D
S3150800B850741100208C0C0020900C002010B5A8B1A3
S3150800B8600446104B1B6843B14FF0500383F311880D
S3150800B870BFF36F8FBFF34F8FFEE7FFF7D9FE0021A7
S3150800B8802046FFF7D3FDFFF76DFF48B94FF0E023D9
S3150800B8904FF08052C3F8042DBFF34F8FBFF36F8F5D
S3150800B8A010BD00BF780C0020224B1B681BB1224B31
S3150800B8B001221A607047204B00221A601F4B1B6832
S3150800B8C003EB83018A001E498A585AB90BB1013B1A
S3150800B8D0F6E74FF0500383F31188BFF36F8FBFF37A
S3150800B8E04F8FFEE7084603EB83018A00024451683E
S3150800B8F04968516003EB830C4FEA8C020832024414
S3150800B90091420FD003EB830291000D4A0A44526814
S3150800B910D1680C4A116009490B60136854330A4A06
S3150800B92013607047486862469100054A0A445060A9
S3150800B930E8E700BF780C00208C0C0020980C00204B
S3150800B940140D002074110020C800002038B50446E4
S3150800B95000F0D8FDE4B1251D2846FEF7E7FEA36AE8
S3150800B9601BB104F11800FEF7E1FE29462348FEF74D
S3150800B970B9FE94F8A430DBB2012B0CD000F0E4FD3C
S3150800B9801F4B1B685BB91F4B1B68A3420ED038BD03
S3150800B9901C4B1C68DFE7002384F8A430EEE700F0B0
S3150800B9A0B1FDFFF7E7FB00F0CFFDECE7144B1B6892
S3150800B9B0B3B1154B1B6843B14FF0500383F311889D
S3150800B9C0BFF36F8FBFF34F8FFEE74FF0E0234FF0C3
S3150800B9D08052C3F8042DBFF34F8FBFF36F8FD6E79E
S3150800B9E0064B1A68094B1B689A4203D1054B00227D
S3150800B9F01A60CCE7FFF758FFC9E700BFA40C002080
S3150800BA00940C002074110020780C0020A00C002053
S3150800BA1058B110B50C46094A11681831FEF76DFE83
S3150800BA2001212046FFF702FD10BD4FF0500383F3B6
S3150800BA301188BFF36F8FBFF34F8FFEE77411002095
S3150800BA4070B110B514460246114B1B688BB94FF0FE
S3150800BA50500383F31188BFF36F8FBFF34F8FFEE751
S3150800BA604FF0500383F31188BFF36F8FBFF34F8FE7
S3150800BA70FEE7084B186841F00041816119681831E2
S3150800BA801046FEF72FFE01212046FFF7CFFC10BD1A
S3150800BA90780C00207411002038B570B10D46144694
S3150800BAA00A4A11681831FEF71DFE0CB14FF0FF3532
S3150800BAB021462846FFF7BAFC38BD4FF0500383F3FA
S3150800BAC01188BFF36F8FBFF34F8FFEE77411002005
S3150800BAD038B5C368DC6824B304F118052846FEF7B0
S3150800BAE025FE184B1B682BBB251D2846FEF71EFE98
S3150800BAF0E06A154B1B68984201D9134B186000EB96
S3150800BB0080002946114B03EB8000FEF7EBFDE26A45
S3150800BB100F4B1B68DB6A9A4211D901200D4B18603E
S3150800BB2038BD4FF0500383F31188BFF36F8FBFF30F
S3150800BB304F8FFEE729460848FEF7D4FDE7E70020C1
S3150800BB40EEE700BF780C0020980C0020140D0020AA
S3150800BB50741100208C0C0020D00C002038B51C4B2A
S3150800BB601B6843B94FF0500383F31188BFF36F8FF7
S3150800BB70BFF34F8FFEE741F000410160C468F4B19E
S3150800BB80FEF7D4FD251D2846FEF7D0FDE06A114BC9
S3150800BB901B68984201D90F4B186000EB80002946B4
S3150800BBA00D4B03EB8000FEF79DFDE26A0B4B1B680D
S3150800BBB0DB6A9A4202D90A4B01221A6038BD4FF055
S3150800BBC0500383F31188BFF36F8FBFF34F8FFEE7E0
S3150800BBD0780C0020980C0020140D00207411002009
S3150800BBE08C0C0020034B1B680360034B1B684360E7
S3150800BBF0704700BF880C00209C0C0020F8B5C8B11F
S3150800BC000C460546F9B100F07DFC1B4B19686B68BC
S3150800BC10C81A2268B2F1FF3F26D0184E36682F6838
S3150800BC20B74201D08B4224D9824215D8002323601B
S3150800BC3001241AE04FF0500383F31188BFF36F8F86
S3150800BC40BFF34F8FFEE74FF0500383F31188BFF31E
S3150800BC506F8FBFF34F8FFEE75B1A134423602846A6
S3150800BC60FFF7C0FF002400E0002400F06DFC20462A
S3150800BC70F8BD0124F9E700BF9C0C0020880C0020C1
S3150800BC80014B01221A6070478C0C0020014B186882
S3150800BC90704700BF74110020054B1B6833B1054B74
S3150800BCA01B680BB1002070470220704701207047BF
S3150800BCB0940C0020780C002000283ED038B50446A5
S3150800BCC0C36A204A1268D26A93422ED28269002A2F
S3150800BCD005DB1C4A1268D26AC2F1380282616169C0
S3150800BCE003EB8303184A02EB8303994205D0154BED
S3150800BCF01B68DB6AE362012038BD251D2846FEF76E
S3150800BD0015FD104B1B68D86AE062104B1B689842F9
S3150800BD1001D90E4B186000EB800029460A4B03EB4D
S3150800BD208000FEF7DFFC0120E6E7C26C054B1B68C6
S3150800BD30DB6A9A4203D30020DEE700207047012021
S3150800BD40DAE700BF74110020140D0020980C0020BB
S3150800BD5000283BD038B504461E4B1B68834208D0E2
S3150800BD604FF0500383F31188BFF36F8FBFF34F8FE4
S3150800BD70FEE7036D43B94FF0500383F31188BFF311
S3150800BD806F8FBFF34F8FFEE7013B0365C16AC26C35
S3150800BD9091421DD00BB1002038BD051D2846FEF77F
S3150800BDA0C5FCE06CE062C0F13803A3610A4B1B686E
S3150800BDB0984201D9084B186000EB80002946074BCA
S3150800BDC003EB8000FEF78EFC0120E5E700207047B4
S3150800BDD00020E1E774110020980C0020140D0020C3
S3150800BDE0002846D038B50446036D43B94FF05003D2
S3150800BDF083F31188BFF36F8FBFF34F8FFEE7C26CD3
S3150800BE008A4200D20A46E16A914201D0012B00D04B
S3150800BE1038BD184B1B68A34222D0E262A369002BE7
S3150800BE2002DBC2F13802A261626901EB8101124BA1
S3150800BE3003EB81039A42EBD1251D2846FEF776FCD3
S3150800BE40E06A0E4B1B68984201D90C4B186000EB50
S3150800BE5080002946084B03EB8000FEF743FCD7E732
S3150800BE604FF0500383F31188BFF36F8FBFF34F8FE3
S3150800BE70FEE7704774110020140D0020980C00206E
S3150800BE80044A136898691368DB6A1268C3F13803B1
S3150800BE909361704774110020054B1B6823B1044B4E
S3150800BEA01A68136D01331365014B1868704700BF94
S3150800BEB074110020064B1A6813682BB90123036016
S3150800BEC023B9D368186870470023F8E7002070473D
S3150800BED07812002008B54160006191420CD8D21A48
S3150800BEE083699A4201D3012008BD011D094B1868D0
S3150800BEF0FEF703FC0020F7E79A4201D2994206D2E0
S3150800BF00011D054B1868FEF7F8FB0020ECE7012039
S3150800BF10EAE700BF741200207812002030B583B01B
S3150800BF2000F0F0FA114B1B681BB100F00DFB03B0D3
S3150800BF3030BD0F4D2846FEF7C7FB0E4C2046FEF7D0
S3150800BF40C3FB0D4B1D600D4B1C60002300930C4B6F
S3150800BF500C4A10210A20FEF7F7FC044B186000284B
S3150800BF60E3D00949FFF7C8F8DFE700BF70120020E1
S3150800BF70901200207C1200207812002074120020F3
S3150800BF8078110020C811002064D200082DE9F0417C
S3150800BF90079F41B94FF0500383F31188BFF36F8FA2
S3150800BFA0BFF34F8FFEE7064614461D4688468FB1F7
S3150800BFB0FFF7B4FF3E60C7F81880FD61069B3B6239
S3150800BFC0381DFEF78CFB2CB197F8283043F0040394
S3150800BFD087F82830BDE8F08110B588B0FFF79EFFD6
S3150800BFE0124B1B68CBB100240594069407AA06A930
S3150800BFF005A8FEF703FA059B0293069B0193022305
S3150800C00000932346079A0A490A48FFF74DFA0A4B4E
S3150800C010186010B1012008B010BD4FF0500383F32B
S3150800C0201188BFF36F8FBFF34F8FFEE770120020A2
S3150800C0306CD20008C9C300086C1200202DE9F04133
S3150800C04082B00446884617461D462C2000F012FC8E
S3150800C050064658B1002380F828300190089B0093C3
S3150800C0602B463A4641462046FFF790FF304602B037
S3150800C070BDE8F08110B584B084462C20039003985F
S3150800C0802C2808D04FF0500383F31188BFF36F8F25
S3150800C090BFF34F8FFEE70398079860B10220079C0D
S3150800C0A084F828000194069800906046FFF76EFF12
S3150800C0B0079804B010BD4FF0500383F31188BFF3FF
S3150800C0C06F8FBFF34F8FFEE7B8B19C4603461848FB
S3150800C0D0006858B300B585B000910192029305290E
S3150800C0E01CDCFFF7D9FD022810D000231A46694642
S3150800C0F00F480068FEF796FC15E04FF0500383F3EF
S3150800C1001188BFF36F8FBFF34F8FFEE70023069AA0
S3150800C110694607480068FEF785FC04E00023624686
S3150800C1206946FEF789FD05B05DF804FB00207047F7
S3150800C1307012002070B582B01B4B1B681A6862B378
S3150800C140DB681E68DC68251D2846FEF7EFFA236AB9
S3150800C1502046984794F8283013F0040FECD0A369CA
S3150800C16033449E4207D26360246129460E4B186801
S3150800C170FEF7C3FAE0E7002100910B463246204657
S3150800C180FFF7A2FF0028D7D14FF0500383F3118899
S3150800C190BFF36F8FBFF34F8FFEE7044A106802495B
S3150800C1A00860136002B070BD781200207412002077
S3150800C1B038B50546FFF744FA0446074B1B68834221
S3150800C1C005D800232B60044B1C60204638BDFFF7BA
S3150800C1D0B1FF01232B60F6E76812002070B582B024
S3150800C1E006460D4617490968C968CC68201DFEF73A
S3150800C1F09DFA94F828C01CF0040F08D12CF0010C05
S3150800C20084F828C0236A2046984702B070BDA16901
S3150800C21033462A4631442046FFF75CFE0028F1D013
S3150800C220002100910B4632462046FFF74DFF0028B5
S3150800C230E8D14FF0500383F31188BFF36F8FBFF334
S3150800C2404F8FFEE77812002070B582B006460C467E
S3150800C250FFF7EEF901A8FFF7ABFF019B33BB0546D5
S3150800C260E4B9B04213D22246711B124B1868FEF786
S3150800C27057FFFFF777FAD8B94FF0E0234FF080520F
S3150800C280C3F8042DBFF34F8FBFF36F8F10E0FFF78E
S3150800C29069FA29463046FFF7A1FF09E0064A1268FF
S3150800C2A012680AB90124DEE71C46DCE7FFF75AFAEA
S3150800C2B002B070BD701200207412002010B588B04C
S3150800C2C002E0049B002B0FDA002204A93D4B1868F4
S3150800C2D0FEF719FD002873D0049B002BF1DA0799A5
S3150800C2E00698059B9847ECE7069C636913B1201DE1
S3150800C2F0FEF71CFA03A8FFF75BFF049B092BE3D89C
S3150800C300DFE803F00505053037500505303794F8A2
S3150800C310283043F0010384F82830059BA1690246BA
S3150800C32019442046FFF7D6FD0028CDD0236A2046BB
S3150800C330984794F8283013F0040FC5D0A269002155
S3150800C34000910B46059802442046FFF7BDFE0028DB
S3150800C350BAD14FF0500383F31188BFF36F8FBFF341
S3150800C3604F8FFEE794F8283023F0010384F828302D
S3150800C370AAE794F8283043F0010384F82830059991
S3150800C380A16131B10346024601442046FFF7A2FDEA
S3150800C3909AE74FF0500383F31188BFF36F8FBFF30B
S3150800C3A04F8FFEE794F8283013F0020F04D023F0DD
S3150800C3B0010384F8283087E7204600F0DDFA83E792
S3150800C3C008B010BD7012002000B583B001A8FFF7B1
S3150800C3D071FD0199FFF738FFFFF770FFF6E740B1E7
S3150800C3E010B5044600F08EF8E46900F0ADF8204672
S3150800C3F010BD4FF0500383F31188BFF36F8FBFF35F
S3150800C4004F8FFEE710B584B014461A466FF0010345
S3150800C410009301900291039400236946024800683C
S3150800C420FEF70AFC04B010BD7012002082B000238B
S3150800C43001930D4B1B68B3F1FF3F08D04FF0500333
S3150800C44083F31188BFF36F8FBFF34F8FFEE74FF06B
S3150800C450500383F31188BFF36F8FBFF34F8F019B90
S3150800C460002BFCD002B07047C400002008480068C2
S3150800C470006880F308884FF0000080F3148862B6DD
S3150800C48061B6BFF34F8FBFF36F8F00DF00BF0000A9
S3150800C49008ED00E0DFF80C00016841F47001016066
S3150800C4A07047000088ED00E04FF0807340F8043CC8
S3150800C4B021F0010140F8081C054B40F80C3C40F8F7
S3150800C4C0202C6FF0020340F8243C4438704700BF24
S3150800C4D02DC4000800000000000000000000000055
S3150800C4E0074B19680868B0E8F04F80F30988BFF36E
S3150800C4F06F8F4FF0000080F311887047AFF300800C
S3150800C500741100204FF0500383F31188BFF36F8F27
S3150800C510BFF34F8F0B4A136801331360012B00D00A
S3150800C52070474FF0E023D3F8043D13F0FF0FF7D020
S3150800C5304FF0500383F31188BFF36F8FBFF34F8F0C
S3150800C540FEE700BFC4000020094B1B6843B94FF043
S3150800C550500383F31188BFF36F8FBFF34F8FFEE746
S3150800C560013B034A13600BB983F31188704700BF78
S3150800C570C4000020000000000000000000000000C9
S3150800C580EFF30980BFF36F8F154B1A681EF0100F73
S3150800C59008BF20ED108A20E9F04F10602DE9090048
S3150800C5A04FF0500080F31188BFF34F8FBFF36F8FA2
S3150800C5B0FFF77AF94FF0000080F3118809BC196873
S3150800C5C00868B0E8F04F1EF0100F08BFB0EC108AEC
S3150800C5D080F30988BFF36F8F704700BFAFF3008001
S3150800C5E07411002008B54FF0500383F31188BFF388
S3150800C5F06F8FBFF34F8FFFF729F828B14FF0E0236D
S3150800C6004FF08052C3F8042D002383F3118808BD28
S3150800C6104FF0E022002313619361054B1B6805491F
S3150800C620A1FB03139B09013B536107231361704761
S3150800C63094000020D34D62104FF0E023D3F8002D6C
S3150800C6403D4B9A421CD04FF0E023D3F8002D3B4BCC
S3150800C6509A421ED030B583B0394B1A78D2B20192BD
S3150800C660FF221A701B78DBB28DF803309DF8033071
S3150800C67003F05003334A1370334B07221A601BE04A
S3150800C6804FF0500383F31188BFF36F8FBFF34F8FBB
S3150800C690FEE74FF0500383F31188BFF36F8FBFF3A4
S3150800C6A04F8FFEE7284A1368013B13609DF8033055
S3150800C6B05B00DBB28DF803309DF8033013F0800F72
S3150800C6C0F0D1214B1B68032B08D04FF0500383F39E
S3150800C6D01188BFF36F8FBFF34F8FFEE71B021A4A0D
S3150800C6E0136003F4E0631360019BDBB2144A137012
S3150800C6F04FF0E024D4F8203D43F47003C4F8203DFD
S3150800C700D4F8203D43F07043C4F8203DFFF780FF7E
S3150800C71000250E4B1D60FFF7BDFED4F8343F43F0ED
S3150800C7204043C4F8343FFFF7A1FEFFF7BDF8FFF713
S3150800C7307DFE284603B030BD71C20F4170C20F415D
S3150800C74000E400E0A8120020A4120020C400002083
S3150800C750EFF305830F2B0FD9114A9B5CDBB2114A05
S3150800C76012789A4208D94FF0500383F31188BFF321
S3150800C7706F8FBFF34F8FFEE74FF0E023D3F80C3DE2
S3150800C78003F4E063084A1268934208D94FF050034D
S3150800C79083F31188BFF36F8FBFF34F8FFEE77047A0
S3150800C7A0F0E300E0A8120020A4120020124A12F0BA
S3150800C7B0070F1ED0D11D21F00701C1F50043134410
S3150800C7C00A460E480260002141601344083B23F0E4
S3150800C7D007030B48036059601960991A5160136082
S3150800C7E0084B1960084B1960084B4FF000421A6055
S3150800C7F070474FF40043E4E7CC120020C41200202F
S3150800C800C0120020B8120020BC120020AC12002072
S3150800C810164B1A461B688342FBD3516802EB010C80
S3150800C820844509D0416800EB010C634509D00360D3
S3150800C830904219D010607047406801445160104614
S3150800C840F0E710B40A4C2468A3420BD05B6819447D
S3150800C850416013681B680360904200D010605DF861
S3150800C860044B70470460F7E7704700BFC412002006
S3150800C870C012002038B50446FEF7DAFE384B1B68AE
S3150800C880B3B1384B1B681C4250D1002C50D004F170
S3150800C890080214F0070F02D022F007020832002A15
S3150800C8A055D0314B1B68934253D330490C6804E08A
S3150800C8B0FFF77CFFE5E721461C466368934202D2F0
S3150800C8C02368002BF7D1264B1B68A34243D00D687B
S3150800C8D0083523680B6063689B1A102B10D9A018BB
S3150800C8E010F0070F08D04FF0500383F31188BFF3F9
S3150800C8F06F8FBFF34F8FFEE743606260FFF788FFD5
S3150800C900626819490B689B1A0B60194909688B42BA
S3150800C91001D217490B60134B1B681343636000234E
S3150800C9202360144A13680133136002E0002500E00F
S3150800C9300025FEF717FF15F0070F0ED04FF050032E
S3150800C94083F31188BFF36F8FBFF34F8FFEE7002580
S3150800C950EFE70025EDE70025EBE7284638BD00BFE1
S3150800C960C0120020AC120020BC120020C412002005
S3150800C970B8120020B4120020002834D038B5044676
S3150800C980A0F1080550F8043C174A1268134208D16A
S3150800C9904FF0500383F31188BFF36F8FBFF34F8FA8
S3150800C9A0FEE750F8081C41B14FF0500383F3118895
S3150800C9B0BFF36F8FBFF34F8FFEE723EA020340F8FA
S3150800C9C0043CFEF735FE54F8041C084A13680B4469
S3150800C9D013602846FFF71CFF054A136801331360E6
S3150800C9E0FEF7C0FE38BD7047AC120020BC1200200E
S3150800C9F0B0120020DFF834D0F8F7C0FC0C480D4917
S3150800CA000D4A002302E0D458C4500433C4188C429B
S3150800CA10F9D30A4A0A4C002301E013600432A24201
S3150800CA20FBD300F06FF8F8F715FAFEE700000120CF
S3150800CA30000000201801002088D2000818010020F4
S3150800CA400C940020FEE702440346934200D1704747
S3150800CA5003F8011BF9E70000294B1B68834270B5F0
S3150800CA6004464BD0C369ABB1DB686BB10025E369FB
S3150800CA70DB68595900293BD10435802DF7D1E36984
S3150800CA802046D96800F072F8E369196811B12046A2
S3150800CA9000F06CF8616911B1204600F067F8E169A9
S3150800CAA011B1204600F062F8216B11B1204600F062
S3150800CAB05DF8616B11B1204600F058F8A16B11B111
S3150800CAC0204600F053F8A16C11B1204600F04EF84C
S3150800CAD0616C11B1204600F049F8E16A11B12046AF
S3150800CAE000F044F8236A4BB12046BDE87040184769
S3150800CAF00E68204600F03AF83146BBE770BD00BF25
S3150800CB00C800002070B50D4D0D4C641BA4100026FE
S3150800CB10A64209D10B4D0C4C00F07EF8641BA410FC
S3150800CB200026A64205D170BD55F8043B9847013644
S3150800CB30EEE755F8043B98470136F2E778D2000845
S3150800CB4078D2000878D200087CD20008704770476F
S3150800CB500A44914200F1FF3300D1704710B511F82D
S3150800CB60014B03F8014F9142F9D110BD38B505467E
S3150800CB70002941D051F8043C0C1F002BB8BFE4181B
S3150800CB8000F03EF81D4A136833B9636014602846FE
S3150800CB90BDE8384000F03AB8A34208D92068211801
S3150800CBA08B4201BF19685B6809182160EDE71A46D0
S3150800CBB05B680BB1A342FAD911685018A0420BD191
S3150800CBC020680144501883421160E0D118685B68F8
S3150800CBD0536008441060DAE702D90C232B60D6E7C5
S3150800CBE0206821188B4204BF19685B68636004BF1C
S3150800CBF0091821605460CAE738BD00BF08940020B0
S3150800CC000148FFF7A3BF00BF049400200148FFF7BF
S3150800CC109EBF00BF04940020F8B500BFF8BC08BC4E
S3150800CC209E467047F8B500BFF8BC08BC9E467047DC
S3150800CC30494E49545F5468726561640030CC0008F7
S3150800CC4000000000000000000000000000000000D6
S3150800CC50000400002F000000000000000000000093
S3150800CC604D41494E5F5761746368646F6700000001
S3150800CC704D41494E5F55706461746554696D6572BE
S3150800CC80000000004D41494E5F4576656E745F466B
S3150800CC906C616773000000004D41494E5F43414E89
S3150800CCA05F52785F51756575650000004D41494EC4
S3150800CCB05F5468726561640060CC0008000000007B
S3150800CCC0000000000000000070CC00080000000012
S3150800CCD0000000000000000084CC000800000000EE
S3150800CCE0000000000000000098CC000800000000CA
S3150800CCF00000000000000000000000000000000026
S3150800CD00ACCC000800000000000000000000000095
S3150800CD1000000000000400002100000000000000E0
S3150800CD20000000005045434F5F4576656E745F46C8
S3150800CD306C616773000000005045434F5F5570648F
S3150800CD4061746554696D6572000000005045434F73
S3150800CD505F5468726561640024CD00080000000015
S3150800CD60000000000000000038CD000800000000A8
S3150800CD7000000000000000004CCD00080000000084
S3150800CD800000000000000000000000000004000091
S3150800CD90280000000000000000000000564152482C
S3150800CDA05F4D7574657800009CCD0008030000008F
S3150800CDB00000000000000000000000000100000064
S3150800CDC00000000001000000010000000000000053
S3150800CDD00000A0C000004041110000000000000053
S3150800CDE0000000000000C84211000000000000001A
S3150800CDF0000000000000C84211000000000000000A
S3150800CE00000000000000C842010000000000B84110
S3150800CE10000020C200004842110000000000204126
S3150800CE20000000000000404111000000000000C0A2
S3150800CE300000A0C00000000009000000000000007B
S3150800CE40000048C200004842090000000000000037
S3150800CE50000048C200004842090000000000000027
S3150800CE60000020C100002041090000000000000069
S3150800CE70000000C100007041090000000000000029
S3150800CE80000020C100002041090000000000000049
S3150800CE90000000000000A04009000000000000009B
S3150800CEA0000048C200001643090000000000000008
S3150800CEB00000A0410000F041090000000000000049
S3150800CEC0000000000000A04009000000000000006B
S3150800CED000000000000016430800000000000000E3
S3150800CEE0000000000100000008000000000000002B
S3150800CEF000000000FFFFFFFF11000000333353401E
S3150800CF000200000000008040414443445F4D7574B0
S3150800CF106578000008CF0008030000000000000044
S3150800CF2000000000414E50495F4D75746578000059
S3150800CF30414E50495F4576656E745F466C6167730E
S3150800CF4000000000414E50495F54687265616400F4
S3150800CF5024CF0008030000000000000000000000C5
S3150800CF6030CF0008000000000000000000000000AC
S3150800CF7044CF000800000000000000000000000088
S3150800CF80000000000004000010000000000000007F
S3150800CF900000000000000000000004419A996D415D
S3150800CFA000000441000020410000A040000020418C
S3150800CFB00000A040414E504F5F4576656E745F464F
S3150800CFC06C61677300000000414E504F5F557064F6
S3150800CFD061746554696D657200000000414E504FDA
S3150800CFE05F54687265616400B4CF000800000000F1
S3150800CFF00000000000000000C8CF00080000000084
S3150800D0000000000000000000DCCF0008000000005F
S3150800D01000000000000000000000000000040000FE
S3150800D020180000000000000000000000000400488E
S3150800D03040000000010000000000000001000000A0
S3150800D0400000000001000000000000000004004885
S3150800D05020000000010000000000000001000000A0
S3150800D0600000000001000000000000000008004861
S3150800D0700040000001000000000000000100000060
S3150800D0800000000000000000010000000000004849
S3150800D090000100000100000000000000010000007F
S3150800D0A00000000000000000010000000004004825
S3150800D0B080000000000000000000000001000000E1
S3150800D0C00000000000000000010000000008004801
S3150800D0D000800000000000000000000001000000C1
S3150800D0E000000000000000000100000000040048E5
S3150800D0F00800000000000000000000000100000019
S3150800D10000000000000000000100000000040048C4
S3150800D11010000000000000000000000001000000F0
S3150800D12000000000000000000100000000000048A8
S3150800D1300080000000000000000000000100000060
S3150800D14000000000000000000100000000030020AD
S3150800D1500000000094D10008010000000200000051
S3150800D160535049445F4576656E745F466C616773D4
S3150800D17000000000535049445F4144435F4D7574B5
S3150800D1806578000060D1000800000000000000007B
S3150800D1900000000074D10008030000000000000031
S3150800D1A00000000054454D505F5468726561640084
S3150800D1B0A4D10008000000000000000000000000E4
S3150800D1C00000000000040000180000000000000035
S3150800D1D0000000005553464C5F4D75746578000095
S3150800D1E0D4D1000803000000000000000000000081
S3150800D1F044656661756C7400F0D100080000000093
S3150800D200000000000000000000000000000200000E
S3150800D210180000000000000000000000A0860100C1
S3150800D220400D0300801A060000350C0040420F002E
S3150800D23080841E0000093D0000127A000024F400D4
S3150800D24000366E010048E801006CDC0200000000B0
S3150800D25000000000010203040607080949444C457A
S3150800D26000000000546D725100000000546D7220D9
S30D0800D27053766300000000007C
S30D0800D278B529000800000000BA
S30D0800D2809129000800000000D6
S3150800D28800FF00000802002010020020000000002D
S3150800D2980000000000000000000000000000000078
S3150800D2A80000000000000000000000000000000068
S3150800D2B80000000000000000000000000000000058
S3150800D2C8000000000060000000000000E0E900001F
S3150800D2D80000000000000000010000000000000037
S3150800D2E801000000010000000000000000400000E6
S3150800D2F80000000000E80000000000000000000030
S3150800D3080000000000000000010000000100000005
S3150800D3180000000000093D000100000010000000A0
S3150800D32800000000000000000000000000000000E7
S3150800D33801000000000000000000000000000000D6
S3150800D34820000000AAAAAAAACC0000200000000013
S3150800D358CC920020349300209C9300200000000003
S3150800D36800000000000000000000000000000000A7
S3150800D3780000000000000000000000000000000097
S3150800D3880000000000000000000000000000000087
S30D0800D39800000000000000007F
S7050800C9F534
